:100000000C94C10C0C94E00C0C94E00C0C94E00CDF
:100010000C94E00C0C94E00C0C94E00C0C94E00CB0
:100020000C94E00C0C94E00C0C94E00C0C94E00CA0
:100030000C94E00C0C94E00C0C94E00C0C941A0F53
:100040000C94E00C0C94E00C0C94EF0E0C94E00C6F
:100050000C94E00C0C94E00C0C949B0F0C94E00CB2
:100060000C94E00C0C94E00C0C94E00C0C94E00C60
:100070000C94E00C0C94E00C0C94E00C0C94E00C50
:100080000C94E00C0C94E00C0C94E00C4C696E6544
:10009000206E756D626572206F7574206F662072B8
:1000A000616E6765000000000000000000000000B5
:1000B0000000000053796E746178206572726F726F
:1000C0000000000000000000000000000000000030
:1000D000000000000000000000000000496E766192
:1000E0006C69642065787072657373696F6E000067
:1000F0000000000000000000000000000000000000
:1001000000000000556E62616C616E636564207072
:100110006172656E730000000000000000000000C6
:100120000000000000000000000000004461746155
:100130002074797065206D69736D61746368000067
:1001400000000000000000000000000000000000AF
:1001500000000000496C6C6567616C206F7065720F
:1001600061746F72000000000000000000000000D9
:10017000000000000000000000000000496C6C65F9
:1001800067616C207661726961626C6500000000D5
:10019000000000000000000000000000000000005F
:1001A00000000000496C6C6567616C20746F6B65C2
:1001B0006E2028696E7465726E616C206572726F54
:1001C0007229000000000000000000004F7574203C
:1001D0006F66206D656D6F72790000000000000091
:1001E000000000000000000000000000000000000F
:1001F00000000000496E7465676572206F76657255
:10020000666C6F7700000000000000000000000036
:10021000000000000000000000000000496E766150
:100220006C696420686578206469676974000000FF
:1002300000000000000000000000000000000000BE
:1002400000000000486578206E756D626572206F51
:10025000766572666C6F7700000000000000000099
:100260000000000000000000000000004D697373F2
:10027000696E672071756F746500000000000000F2
:10028000000000000000000000000000000000006E
:10029000000000004578706563746564206F7065C8
:1002A0006E206F7220636C6F736520706172656E73
:1002B000000000000000000000000000274F4E2753
:1002C0002073796E746178206572726F720000001D
:1002D000000000000000000000000000000000001E
:1002E000000000004D697373696E67205448454EE5
:1002F00020696E2049462073746174656D656E7463
:100300000000000000000000000000004D69737351
:10031000696E6720544F20696E20464F52207374D7
:100320006174656D656E74000000000000000000DF
:10033000000000004C696E65206E756D626572206C
:100340006572726F72000000000000000000000083
:10035000000000000000000000000000496C6C6517
:1003600067616C20646174612074797065000000BD
:10037000000000000000000000000000000000007D
:100380000000000045787072657373696F6E2074A9
:100390006F6F20636F6D706C657800000000000067
:1003A0000000000000000000000000004D697373B1
:1003B000696E6720636F6D6D6100000000000000D2
:1003C000000000000000000000000000000000002D
:1003D000000000004D697373696E6720636F6D6D77
:1003E00061206F722073656D69636F6C6F6E0000C2
:1003F0000000000000000000000000004D61746873
:1004000020737461636B206F766572666C6F770022
:1004100000000000000000000000000000000000DC
:1004200000000000556E64696D656E73696F6E65DE
:100430006420617272617900000000000000000019
:10044000000000000000000000000000537562730F
:100450006372697074206F7574206F662072616EAC
:1004600067650000000000000000000000000000C0
:1004700000000000446976696465206279207A652D
:10048000726F00000000000000000000000000008B
:100490000000000000000000000000004C696E65D4
:1004A000206E6F7420666F756E640000000000009F
:1004B000000000000000000000000000000000003C
:1004C00000000000546F6F206D616E79206E6573BF
:1004D00074656420474F53554273000000000000CC
:1004E00000000000000000000000000052455455CC
:1004F000524E20776974686F757420474F53554288
:1005000000000000000000000000000000000000EB
:1005100000000000546F6F206D616E79206163747C
:10052000697665205748494C45730000000000007B
:10053000000000000000000000000000454E44578D
:100540004820776974686F7574205748494C450096
:10055000000000000000000000000000000000009B
:10056000000000004F4E20617267756D656E74204B
:100570006D757374206265203E207A65726F00008D
:100580000000000000000000000000004E6F6E73CD
:100590007562736372697074207661726961626CEE
:1005A0006520696E2044494D0000000000000000F5
:1005B000000000005661726961626C6520616C72B6
:1005C000656164792044494D656E73696F6E656439
:1005D000000000000000000000000000546F6F20C9
:1005E0006D616E792061637469766520464F522D86
:1005F0004E455854206C6F6F70730000000000006F
:10060000000000004E45585420646F6573206E6FE3
:1006100074206D6174636820464F52000000000032
:1006200000000000000000000000000043616E2791
:100630007420434F4E54696E756500000000000041
:1006400000000000000000000000000000000000AA
:10065000000000004F7574206F6620646174612093
:10066000696E2052454144206F7220524553544FC9
:100670005245000000000000000000004E65676168
:100680007469766520737562736372697074206E25
:100690006F7420616C6C6F7765640000000000006F
:1006A00000000000496C6C6567616C20454550286E
:1006B0002920617267756D656E740000000000008E
:1006C0000000000000000000000000004F6E6C7988
:1006D00020616C6C6F77656420696E205052494EC2
:1006E000542073746174656D656E740000000000C1
:1006F00000000000417267756D656E74206F75743F
:10070000206F662072616E676520696E20544142D9
:10071000000000000000000000000000546F6F2087
:100720006D616E7920617267756D656E7473206995
:100730006E2043414C4C000000000000000000000F
:1007400000000000417275676D656E7420746F2043
:1007500074696D6524282920697320756E6B6E6F2E
:10076000776E000000000000000000002D2D2034F6
:1007700035202D2D000000000000000000000000CA
:100780000000000000000000000000000000000069
:10079000000000002D2D203436202D2D00000000FB
:1007A0000000000000000000000000000000000049
:1007B0000000000000000000000000002D2D20348B
:1007C00037202D2D00000000000000000000000078
:1007D0000000000000000000000000000000000019
:1007E000000000002D2D203438202D2D00000000A9
:1007F00000000000000000000000000000000000F9
:100800000000000000000000000000002D2D20343A
:1008100039202D2D00000000000000000000000025
:1008200000000000000000000000000000000000C8
:10083000000000002D2D203530202D2D000000005F
:1008400000000000000000000000000000000000A8
:100850000000000000000000000000002D2D2035E9
:1008600031202D2D000000000000000000000000DD
:100870000000000000000000000000000000000078
:10088000000000002D2D203532202D2D000000000D
:100890000000000000000000000000000000000058
:1008A0000000000000000000000000002D2D203599
:1008B00033202D2D0000000000000000000000008B
:1008C0000000000000000000000000000000000028
:1008D000000000002D2D203534202D2D00000000BB
:1008E0000000000000000000000000000000000008
:1008F0000000000000000000000000004E6F7420A7
:10090000656E6F75676820454550524F4D20666F84
:100910007220736176650000000000000000000096
:1009200000000000537461636B20756E646572662D
:100930006C6F770000000000000000000000000065
:100940000000000000000000000000005573657208
:1009500020656E746572656420425245414B00000B
:100960000000000000000000000000000000000087
:100970000000000043616E277420757365204144B8
:100980004452207769746820636F6E7374616E746B
:100990000000000000000000000000004E6F742006
:1009A000656E6F75676820666C61736820666F722C
:1009B0002073617665000000000000000000000068
:1009C0000000000020000000000000000000000007
:1009D0000000000000000000000000000000000017
:1009E00000000000000000000000000000002000E7
:1009F00000000000000000007839636872240000E5
:100A000000000000F33373717274000000000000F6
:100A10005B35616273000000000000009633726E67
:100A200064000000000000002C3573676E000000B9
:100A300000000000833974616200000000000000C3
:100A40000000200000000000000000000C35706570
:100A5000656B000000000000CD346565700000008B
:100A6000000000002C3968657800000000000000DC
:100A70000000200000000000000000006D396865E3
:100A800078320000000000005239686578340000B8
:100A900000000000EF347065656B31360000000027
:100AA000D1347065656B3332000000002935616414
:100AB0006472000000000000C934656570313600C2
:100AC00000000000C534656570333200000000008E
:100AD00000002000000000000000000029386C65C4
:100AE0007400000000000000293800000000000031
:100AF000000000008E397072696E74000000000002
:100B0000C73D666F72000000000000008E3B6E65FE
:100B10007874000000000000FB3874726F6E0000F3
:100B200000000000FF3874726F666600000000006D
:100B3000D936706F6B65000000000000293A6469C7
:100B40006D00000000000000773672656D00000047
:100B50000000000000002000000000000000000075
:100B6000833664617461000000000000513D7265CD
:100B70006164000000000000D33A726573746F7204
:100B8000650000000000676F7375620000000000E0
:100B90000000280000000000000000000000290004
:100BA0000000000000000000D037676F746F000085
:100BB00000000000D8366F6E00000000000000004A
:100BC000C13672657475726E00000000643C69661F
:100BD00000000000000000007F3D696E7075740029
:100BE00000000000AC3773746F700000000000005C
:100BF0004937656E64000000000000005C377768CC
:100C0000696C650000000000DA36656E6477680084
:100C100000000000603C65657000000000000000FE
:100C20005C3C65657031360000000000583C65652D
:100C300070333200000000000000200000000000BF
:100C40000000000000002000000000000000000084
:100C5000B831616E6400000000000000DA316F728C
:100C60000000000000000000FC31656F7200000011
:100C7000000000006E3B696E627974650000000040
:100C8000000020000000000000000000C53A6F6E68
:100C900074696D6500000000C63A6F6E697271007C
:100CA00000000000C73A726574690000000000008F
:100CB000C83A6F6E70616363000000000239736CA4
:100CC00065657000000000000000200000000000CA
:100CD00000000000000020000000000000000000F4
:100CE00000002000000000000000000000002000C4
:100CF00000000000000000000000200000000000D4
:100D000000000000000020000000000000000000C3
:100D1000F8303C000000000000000000CC303E0035
:100D20000000000000000000A0303C3D000000007A
:100D30000000000074303E3D000000000000000094
:100D400048303D0000000000000000001C303C3E28
:100D50000000000000000000000020000000000073
:100D6000000000000000746F0000000000000000A0
:100D700000007468656E0000000000000000656CF3
:100D800073650000000000000000737465700000CF
:100D90000000000000002000000000000000000033
:100DA0000000200000000000000000000000200003
:100DB0000000000000000000000020000000000013
:100DC0000000000000002000000000000000000003
:100DD00096312B00000000000000000074312D004F
:100DE000000000000000000000002B0000000000D8
:100DF000000000008E393F000000000000000000ED
:100E000077362700000000000000000000002000EE
:100E100000000000000000000000200000000000B2
:100E200000000000000020000000000000000000A2
:100E30000000200000000000000000000000200072
:100E40000000000000000000000020000000000082
:100E50000000000000002000000000000000000072
:100E60000000200000000000000000000000200042
:100E70000000000000000000000020000000000052
:100E80000000000000002000000000000000000042
:100E900024312A00000000000000000025322F004D
:100EA00000000000000000004C316D6F6400000085
:100EB0000000000000002000000000000000000012
:100EC00000002000000000000000000000002000E2
:100ED00000000000000000000000200000000000F2
:100EE00000000000000020000000000000000000E2
:100EF00000002000000000000000000000002000B2
:100F000000000000000000000000200000000000C1
:100F100000000000000020000000000000000000B1
:100F20000000200000000000000000000000200081
:100F30000000000000000000000020000000000091
:100F40000000000000002000000000000000000081
:100F5000B12F5E0000000000000000000000200033
:100F60000000000000000000000020000000000061
:100F70000000000000002000000000000000000051
:100F80000000200000000000000000000000200021
:100F90000000000000000000000020000000000031
:100FA0000000000000002000000000000000000021
:100FB00000002000000000000000000000002000F1
:100FC0000000000000000000000020000000000001
:100FD00000000000000020000000000000000000F1
:100FE00000002000000000000000000000002000C1
:100FF00000000000000000000000200000000000D1
:1010000000000000000020000000000000000000C0
:10101000222F40000000000000000000722F6E6FC1
:1010200074000000000000008F2F2D000000000061
:1010300000000000DA2E4033320000000000000003
:101040004A2F403136000000000000000000200060
:101050000000000000000000000020000000000070
:101060000000000000002000000000000000000060
:1010700000002300000000000000000000003D0010
:101080000000000000000000D0263A000000000030
:101090000000000000003B00000000000000000015
:1010A00000002C00000000000000000000002000F4
:1010B0000000000000000000000020000000000010
:1010C0000000000000002000000000000000000000
:1010D00074696D657230000000000000000000F0CF
:1010E000FF0474696D6572310000000000000000AB
:1010F00000F1FF0474696D657232000000000000A9
:10110000000000F2FF0474696D6572330000000096
:101110000000000000F3FF04665F637075000000CC
:1011200000000000000000F4FF04706F72746100A2
:101130000000000000000000003B0001706F7274AE
:101140006200000000000000000000380001706F25
:101150007274630000000000000000000035000110
:10116000706F727464000000000000000000003224
:1011700000016464726100000000000000000000D3
:10118000003A000164647262000000000000000088
:10119000000000370001646472630000000000007A
:1011A000000000000034000164647264000000006C
:1011B0000000000000000031000170696E61000055
:1011C00000000000000000000039000170696E623C
:1011D00000000000000000000000003600017069FF
:1011E0006E630000000000000000000000330001FA
:1011F00070696E6400000000000000000000003014
:10120000000161646373726100000000000000006F
:101210000026000161646D75780000000000000088
:101220000000002700016164636C00000000000002
:1012300000000000002400016164636800000000F9
:101240000000000000000025000161646300000050
:1012500000000000000000000024000273707372A0
:1012600000000000000000000000002E000173706C
:10127000647200000000000000000000002F000168
:101280007370637200000000000000000000002D79
:101290000001757074696D650000000000000000B9
:1012A00000FFFF04706F7274650000000000000012
:1012B000000000230001706F7274660000000000DF
:1012C0000000000000620001706F7274670000008F
:1012D0000000000000000065000164647265000009
:1012E000000000000000000000220001646472663B
:1012F00000000000000000000000006100016464C4
:10130000726700000000000000000000006400019F
:1013100070696E6500000000000000000000002100
:10132000000170696E66000000000000000000000F
:101330000020000170696E670000000000000000DE
:101340000000006300010000000000000000000039
:10135000000000000000000000000000000000008D
:1013600000000000000000000000000A0D6F722065
:101370002765652720746F206C6F61642066726F2B
:101380006D20454550524F4D2E00556E6B6E6F7758
:101390006E20617267756D656E7420746F204C4F9E
:1013A00041443B207573652027666C3C6E3E2720C8
:1013B000746F206C6F61642066726F6D20464C41C3
:1013C00053480020646174612062797465732066FB
:1013D000726F6D20454550524F4D2E002070726F38
:1013E0006772616D20627974657320616E6420009C
:1013F0004C6F616465642000546869732077696C80
:101400006C206F76657277726974652074686520E8
:1014100063757272656E742070726F6772616D2091
:10142000696E2052414D21202041726520796F75EF
:1014300020737572653F20000A0D4E6F2070726F29
:101440006772616D20736176656420696E20454521
:1014500050524F4D21002E004E6F2073756368204F
:10146000666C6173682066696C653B206D7573748A
:10147000206265203020746F20002E00206461748B
:10148000612062797465732066726F6D20666C618D
:1014900073682066696C6520002070726F677261E6
:1014A0006D20627974657320616E6420004C6F61F9
:1014B0006465642000546869732077696C6C206FE0
:1014C00076657277726974652074686520637572D9
:1014D00072656E742070726F6772616D2120204199
:1014E000726520796F7520737572653F20000A0D53
:1014F0004E6F2070726F6772616D207361766564E4
:1015000020696E20666C6173682066696C652000D6
:101510000A0D6F72202765652720746F207361762E
:101520006520746F20454550524F4D2E00556E6B0F
:101530006E6F776E20617267756D656E7420746F63
:1015400020534156453B207573652027666C3C6EE1
:101550003E2720746F207361766520746F20464C9F
:10156000415348004E6F2070726F6772616D206941
:101570006E2052414D3B206E6F7468696E67207318
:10158000617665642E0020646174612062797465FF
:101590007320746F20454550524F4D2E00207072BD
:1015A0006F6772616D20627974657320616E64206B
:1015B0000053617665642000546869732077696C14
:1015C0006C206572617365207468652070726F6746
:1015D00072616D206E6F7720696E20454550524FC5
:1015E0004D21202041726520796F752073757265D9
:1015F0003F200020646174612062797465732074F7
:101600006F20666C6173682066696C6520002070CD
:10161000726F6772616D20627974657320616E64A8
:1016200020005361766564200021202041726520EE
:10163000796F7520737572653F2000546869732057
:1016400077696C6C206572617365207468652070C1
:10165000726F6772616D206E6F7720696E20666CA5
:101660006173682066696C652000206D61726B652E
:101670006420666F72206175746F73746172742E6A
:101680000050726F6772616D20696E20666C6173C5
:10169000682066696C6520000A0D4E6F2070726FBD
:1016A0006772616D20736176656420696E20666C77
:1016B0006173682066696C65200050726F677261A3
:1016C0006D20696E20454550524F4D206D61726B03
:1016D000656420666F72206175746F7374617274D3
:1016E0002E004E6F2070726F6772616D207361768D
:1016F000656420746F20454550524F4D210041755F
:10170000746F737461727420666C61672072656DAA
:101710006F7665642E000A0D4B4C4261736963203D
:10172000666F722041746D656C20415652204154A1
:101730006D6567613132382076302E38000A0D43EE
:101740006F7265207772697474656E206279204BC0
:1017500061726C204C756E742C206261736564201C
:101760006F6E20476F72646F6E20446F7567686D8F
:10177000616E27732042415349433131000A0D4BBA
:101780004C426173696320636F72652076302E3935
:10179000000A0D5245414459003A20004552524F2B
:1017A000522023005E5E5E003A200020696E206CAD
:1017B000696E6520004552524F522023000A0D4E9B
:1017C0006F2070726F6772616D20696E206D656D3C
:1017D0006F72792E000A0D50726F6772616D20650D
:1017E00072617365642E000A0D546869732077690D
:1017F0006C6C206572617365207468652063757216
:1018000072656E742070726F6772616D2120204165
:10181000726520796F7520737572653F20004E6F79
:101820002070726F6772616D206C6F6164656420F7
:10183000696E206D656D6F72792E0A0D006461749A
:101840006100270072656D004E6F2073756368201C
:10185000666C6173682066696C652E00204E6F208F
:1018600070726F6772616D2E003A2000666C002006
:10187000627974657320667265650044796E616D86
:101880006963206D656D6F727920706F6F6C2028B1
:10189000617272617973293A2000206279746573EC
:1018A0002066726565005661726961626C65206DC3
:1018B000656D6F72793A20002062797465732066D5
:1018C0007265650050726F6772616D206D656D6F36
:1018D00072793A2000556E6B6E6F776E20415554C9
:1018E0004F535420617267756D656E742E20204DC4
:1018F000757374206265204F46462C2045452C2088
:10190000464C302C20464C312C206F7220464C32F5
:101910002E00496C6C6567616C206175746F73741F
:101920006172742076616C756520004175746F7307
:10193000746172742066726F6D20666C61736820CA
:10194000004175746F73746172742066726F6D20DC
:10195000454550524F4D2E004175746F737461723E
:1019600074206E6F7420656E61626C65642E000A6F
:101970000D53746F70706564206174206C696E65BE
:10198000200011241FBECFEFD0E1DEBFCDBF13E09A
:10199000A0E0B1E0E4EDFEE700E00BBF02C007907D
:1019A0000D92A431B107D9F71FE0A4E1B3E001C063
:1019B0001D92AC3FB107E1F70E94F9170C94683F04
:1019C0000C9400002CE73EE03093C0052093BF0547
:1019D00030934F0F20934E0F83E49FE090934C0C75
:1019E00080934B0CF90101C0119280914B0C9091A6
:1019F0004C0C8E179F07C0F786E696E09093570C25
:101A00008093560C909373058093720581E49CE05B
:101A10009093450C8093440C08959C01220F331F32
:101A2000F90143E0EE0FFF1F4A95E1F7E20FF31FC4
:101A3000E152FF4E65917491CB014096049750F4AA
:101A4000862F8F7090E0880F991F880F991F875EEF
:101A50009C4F06C08FEF6F3F780741F485E193E01C
:101A60009C01442737FD4095542F0CC08FEF643FF5
:101A7000780729F420E030E040E050E003C09B010B
:101A800040E050E0B901CA0108959C012458314F4B
:101A9000C9010895FC01DB018CEE9CE091838083F9
:101AA00080E991E08D939C930895FC01108211824E
:101AB000128260E070E080E090E008950895FC01FB
:101AC00081E08783838381E090E09187808714821F
:101AD00080E790E09683858360E070E080E090E0AE
:101AE000089508955D9BFECF8DE08CB95D9BFECF80
:101AF0008AE08CB90895982F882391F1809114037E
:101B0000882329F19636E1F0973638F4923681F041
:101B1000953651F09136A9F40DC0923779F094378B
:101B200029F09E3671F408C09BE10BC099E009C012
:101B300098E007C097E005C09AE003C09DE001C0AF
:101B40009CE0109214035D9BFECF9CB908959C35D8
:101B500021F481E08093140308955D9BFECF9CB92E
:101B60000895CF93DF93EC0102C00E947B0DFE012C
:101B7000219684918823C9F7DF91CF91089586E15A
:101B800097E10E94B10D0895CF93DF93EC0102C05D
:101B90000E947B0D89918823D9F7DF91CF91089519
:101BA0005D9BFECF8CB908959091490380914A03C3
:101BB0009817D1F3F894E0914A03F0E0E75DFC4F09
:101BC000808120914A0330E02F5F3F4F2F713070AA
:101BD00020934A0378940895FF920F931F93CF9315
:101BE000DF93EC0110E008E060E2F62E0E94D40DD5
:101BF0008D3079F488835D9BFECF8AE08CB95D9B44
:101C0000FECF8DE08CB9DF91CF911F910F91FF90A6
:101C10000895883071F4112349F35D9BFECF0CB910
:101C20005D9BFECFFCB85D9BFECF0CB92197115098
:101C3000DDCF8A30D9F25D9BFECF8CB989931F5FCF
:101C4000D5CF1F93142FFC01EE0FFF1F9F0143E020
:101C5000220F331F4A95E1F7E20FF31FEF51FF4EBA
:101C600044919C01220F331FF901B3E0EE0FFF1FD7
:101C7000BA95E1F7E20FF31FE152FF4EA591B4913F
:101C8000413011F41C931CC0423031F4812F952F48
:101C900011969C938E9314C0CD014096049780F4C6
:101CA000F894EA2FF0E0EF70F070EE0FFF1FEE0FE8
:101CB000FF1FE75EFC4F1083518362837383789428
:101CC0001F910895FC01EE0FFF1F9F0143E0220FBB
:101CD000331F4A95E1F7E20FF31FEF51FF4E449196
:101CE0009C01220F331FF90183E0EE0FFF1F8A953D
:101CF000E1F7E20FF31FE152FF4EA591B49141309D
:101D000021F48C91282F30E005C0423031F48D91C0
:101D10009C919C0140E050E030C0CD01409604977A
:101D200078F4EA2FF0E0EF70F070EE0FFF1FEE0F87
:101D3000FF1FE75EFC4F20813181428153811DC02E
:101D40008FEFAF3FB80749F4209115033091160388
:101D5000409117035091180310C0A45FBF4F29F0A2
:101D600020E030E040E050E008C020915F03309177
:101D700060034091610350916203B901CA01089563
:101D8000833028F020E030E040E050E010C0E82F41
:101D9000F0E0EE0FFF1FEE0FFF1FEE5FFE4F8081A2
:101DA0009181A0E0B0E02227382F492F5A2FB901A6
:101DB000CA010895CF93DF93EC01A0E0B0E009C021
:101DC0006BBFFA01879189934F5F5F4F6F4F7F4FD2
:101DD0001196A217B307A0F3DF91CF9108951F9238
:101DE0000F920FB60F920BB60F9211248F939F9301
:101DF000EF93FF938CB1833021F481E08093510CF9
:101E00000EC0E0914903F0E0E75DFC4F80838091D4
:101E1000490390E001968F71907080934903FF9180
:101E2000EF919F918F910F900BBE0F900FBE0F906F
:101E30001F9018951F920F920FB60F9211248F9337
:101E40009F93AF93BF938091150390911603A09138
:101E50001703B09118030196A11DB11D80931503BE
:101E600090931603A0931703B0931803809119035E
:101E700090911A03A0911B03B0911C030097A10538
:101E8000B10559F00197A109B10980931903909305
:101E90001A03A0931B03B0931C0380911D03909120
:101EA0001E03A0911F03B09120030097A105B10567
:101EB00059F00197A109B10980931D0390931E0366
:101EC000A0931F03B09320038091210390912203DC
:101ED000A0912303B09124030097A105B10559F007
:101EE0000197A109B1098093210390932203A09344
:101EF0002303B09324038091250390912603A0919E
:101F00002703B09128030097A105B10559F0019767
:101F1000A109B1098093250390932603A093270379
:101F2000B0932803BF91AF919F918F910F900FBEF7
:101F30000F901F9018951F920F920FB60F921124B9
:101F40000F900FBE0F901F9018959B01BC01660F5C
:101F5000771FCB01E3E0880F991FEA95E1F7680F3F
:101F6000791F60537F4EC9010E942E3F0895CF9282
:101F7000DF92EF92FF920F931F93DF93CF93CDB732
:101F8000DEB72F970FB6F894DEBF0FBECDBFFF248C
:101F9000A2E1EA2E6E010894C11CD11CFE9C8001B6
:101FA000112400531F4EC8010E94353F892B59F060
:101FB000C601B8010E942E3FC6010E946B19892BF1
:101FC000A1F4F394EBCF20E030E0C9012F960FB6D7
:101FD000F894DEBF0FBECDBFCF91DF911F910F915F
:101FE000FF90EF90DF90CF900895E091520CF09128
:101FF000530C83E88193F093530CE093520C8F2D94
:1020000090E00E94BD1821E030E0DFCFCF93DF9356
:102010000E947718E0915B0CF0915C0C808190E05D
:10202000C0970A9718F0C0E0D0E036C020E030E05A
:1020300011C0C90163E0880F991F6A95E1F7220F6B
:10204000331F280F391F240F351F3196F0935C0C76
:10205000E0935B0CE0915B0CF0915C0C8081482F6D
:1020600050E0405350404A30510518F3E9010E94B6
:102070007718C330D10584F088E594E10E94B10D52
:1020800062E070E080E090E00E947F2186E594E1CC
:102090000E94B10DCFEFDFEFCE01DF91CF91089518
:1020A0008F929F92AF92BF92CF92DF92EF92FF9268
:1020B0000F931F93CF93DF934C01FC01EE0FFF1F93
:1020C000EE0FFF1FE050FF4F80819181A0E0B0E054
:1020D000EE24F82E092F1A2F7CE0A72EB12CC12C4C
:1020E000D12CAE0CBF1CC01ED11ECBBEF5018791FA
:1020F00096918F5F9F4F61F48EEE94E10E94B10D37
:10210000B401882777FD8095982F0E947F2121C1F7
:102110002091560C3091570C809172059091730567
:102120002817390789F085EB94E10E94B10D8BE403
:1021300093E00E94EC0D80914B0390E00E941E3FC3
:102140008937910509F005C1CBBEF501A791B6917C
:10215000AA59B94FB093570CA093560C4EE050E0DB
:1021600060E070E0E40EF51E061F171F0BBFF701BD
:10217000479156914A0F5B1F509373054093720528
:1021800062E070E080E090E0E60EF71E081F191F85
:102190000BBFF701879196918458914F9093C0059A
:1021A0008093BF0562E0A62EB12CC12CD12CEA0C85
:1021B000FB1C0C1D1D1D0BBFF70127913691820FD3
:1021C000931F90934F0F80934E0F64E070E080E078
:1021D00090E0E60EF71E081F191F0BBFF70187914D
:1021E00096918451934F9093B8058093B7055A0107
:1021F000AA1ABB0AF401EE0FFF1FEE0FFF1FEE5FDE
:10220000FE4F808191817C0100E010E0502F4F2D26
:102210003E2D222760E070E016C04BBFF901879188
:102220008C932F5F3F4F4F4F5F4F222349F4089409
:10223000E11CF11C011D111D502F4F2D3E2D222799
:1022400011966F5F7F4F6A157B0538F30894E11C88
:10225000F11C011D111D502F4F2D3E2D2227A09145
:10226000BF05B091C005C0904E0FD0904F0FCA1A55
:10227000DB0A60E070E016C04BBFF90187918C93D8
:102280002F5F3F4F4F4F5F4F222349F40894E11CCB
:10229000F11C011D111D502F4F2D3E2D222711968F
:1022A0006F5F7F4F6C157D0538F30894E11CF11CBE
:1022B000011D111D502F4F2D3E2D2227C091B70516
:1022C000D091B805CC5EDC40ACEEBCE060E070E0E4
:1022D00016C04BBFF90187918C932F5F3F4F4F4F33
:1022E0005F4F222349F40894E11CF11C011D111DCC
:1022F000502F4F2D3E2D222711966F5F7F4F6C1769
:102300007D0738F30E948F2D9093510F8093500FCB
:102310008DEA94E10E94B10DB50180E090E00E9449
:102320007F2189E994E10E94B10DB60180E090E03F
:102330000E947F218CE794E10E94B10DB4018827AF
:1023400077FD8095982F0E947F218AE794E10E9473
:10235000B10DDF91CF911F910F91FF90EF90DF9022
:10236000CF90BF90AF909F908F900895EF92FF9283
:102370000F931F937C010E94503F182F00E0C7016C
:1023800001960E94503F080F111DC8011F910F9127
:10239000FF90EF900895AF92BF92CF92DF92EF92AD
:1023A000FF920F931F93CF93DF938CE090E00E94F6
:1023B000B6118F5F9F4F19F488E394E191C020918B
:1023C000560C3091570C8091720590917305281727
:1023D000390789F088EF93E10E94B10D8BE493E017
:1023E0000E94EC0D80914B0390E00E941E3F8937C4
:1023F000910509F077C08CE090E00E94B611B6E636
:10240000CB2EB6E0DB2EC80ED91ED092570CC09250
:10241000560C8EE090E00E94B6117601E80EF91E8F
:10242000F0927305E092720580E190E00E94B6118F
:102430008C010458114F1093C0050093BF0582E131
:1024400090E00E94B611080F191F10934F0F0093D0
:102450004E0F5701AC18BD08C0E0D0E008C0CE0157
:102460004A960E94503FF60181936F012196CA154A
:10247000DB05A8F3E090BF05F090C005C0904E0FBB
:10248000D0904F0FCE18DF088501065E1F4FC0E0C9
:10249000D0E009C0C8010E94503FF70181937F013D
:1024A00021960F5F1F4FCC15DD05A0F30E948F2DE5
:1024B0009093510F8093500F80EF93E10E94B10DE4
:1024C000B50180E090E00E947F218CED93E10E94B5
:1024D000B10DB60180E090E00E947F2183EC93E192
:1024E0000E94B10DDF91CF911F910F91FF90EF905E
:1024F000DF90CF90BF90AF9008950F931F93CF932D
:10250000DF930E94771800915B0C10915C0CF8012E
:1025100080818D3071F090E00E941E3F85369105DC
:1025200059F4F801818190E00E941E3F85369105A3
:10253000F1F40E94CB1123C086369105C1F4E80165
:102540002196F801818190E00E941E3F8C36910512
:1025500071F42196D0935C0CC0935B0C0E94061022
:10256000FFEF8F3F9F0759F00E94501008C08AE884
:1025700093E10E94B10D8BE693E10E94B10DDF91D2
:10258000CF911F910F91089588E190E00E94503FF4
:10259000089588E190E00E94503F8A3579F08B35AC
:1025A00018F4853529F407C08B3559F08C3561F066
:1025B00020E030E00FC00E94CB110AC080E090E024
:1025C00005C081E090E002C082E090E00E945010DF
:1025D00021E030E0C9010895CF92DF92EF92FF929F
:1025E0000F931F93DC01CB016C010E94503FE82E3A
:1025F000FF2400E010E0102F0F2DFE2CEE24C6016A
:1026000001960E94503FE80EF11C011D111DB701FB
:10261000C8011F910F91FF90EF90DF90CF90089528
:10262000AF92BF92CF92DF92EF92FF920F931F93E0
:102630007B018C010E94EC125B016C016501BB24E3
:10264000AA2482E090E0A0E0B0E0E80EF91E0A1FA4
:102650001B1FC801B7010E94EC129B01AC012A0D9F
:102660003B1D4C1D5D1DB901CA011F910F91FF90CB
:10267000EF90DF90CF90BF90AF900895AF92BF9250
:10268000CF92DF92EF92FF920F931F931092490324
:1026900010924A031092510C60E070E080E090E0EC
:1026A0000E9410137B018C0160935F0370936003A1
:1026B000809361039093620364E070E080E090E0B7
:1026C0000E9410135B016C016093630370936403B9
:1026D000809365039093660368E070E080E090E08B
:1026E0000E941013AE0CBF1CC01ED11EA616B7064A
:1026F000C806D906C1F080E094E2A4EFB0E0809370
:102700005F0390936003A0936103B093620380E042
:1027100096E9A0E0B0E08093630390936403A093F4
:102720006503B093660382E08BB988E98AB976E0E5
:10273000D72ED0929500E0905F03F0906003009157
:10274000610310916203209163033091640340910F
:1027500065035091660363E0220F331F441F551F2A
:102760006A95D1F7C801B7010E94CD3E2150109261
:10277000900029B9D3BEC801B70120E038EE43E08C
:1027800050E00E94CD3E215021BF87B7826087BFB5
:102790001092190310921A0310921B0310921C033B
:1027A00010921D0310921E0310921F03109220031B
:1027B00010922103109222031092230310922403FB
:1027C00010922503109226031092270310922803DB
:1027D00078941F910F91FF90EF90DF90CF90BF9072
:1027E000AF900895DC01CB010E94503F682F70E04C
:1027F00080E090E008951F93CF93DF93EC01162FB4
:102800000E94503F181721F0CE01612F0E94583FBF
:10281000DF91CF911F910895FF920F931F938C0129
:10282000F62E672F0E94FB13C80101966F2D0E94A0
:10283000FB131F910F91FF9008958F929F92AF927B
:10284000BF92CF92DF92EF92FF920F931F93DF938D
:10285000CF93CDB7DEB764970FB6F894DEBF0FBE47
:10286000CDBF8CE090E00E94B6118F5F9F4F81F04A
:1028700088EB95E10E94B10DCE0101960E94EC0D0E
:10288000898190E00E941E3F8937910509F09CC024
:1028900080917205909173052091560C3091570CE0
:1028A000821B930B20914E0F30914F0F4091BF052B
:1028B0005091C005241B350B820F931F4A96875EEB
:1028C0009F4030F087E38093460C0E94F9217CC042
:1028D00088E190E06FEF0E94FB138CE090E060E0F5
:1028E00070E00E940C1460917205709173058091E4
:1028F000560C9091570C681B790B8EE090E00E946B
:102900000C1480E190E060E070E00E940C14609193
:102910004E0F70914F0F8091BF059091C005681BBD
:10292000790B82E190E00E940C14E090560CF0903C
:10293000570C80907205909073058E189F0800E0E8
:1029400010E009C0C8014A96F70161917F010E9419
:10295000FB130F5F1F4F08151905A0F3C090BF05AB
:10296000D090C005A0904E0FB0904F0FAC18BD088E
:10297000EAE1EE2EF12CE80CF91C00E010E00BC0AF
:10298000C701F60161916F010E94FB130F5F1F4F9A
:102990000894E11CF11C0A151B0590F381EB95E1ED
:1029A0000E94B10DB40180E090E00E947F218DE98A
:1029B00095E10E94B10DB50180E090E00E947F2179
:1029C00086E895E10E94B10D64960FB6F894DEBFDB
:1029D0000FBECDBFCF91DF911F910F91FF90EF9070
:1029E000DF90CF90BF90AF909F908F900895CF923F
:1029F000DF92EF92FF920F931F93CF93DF9320917B
:102A0000560C3091570C80917205909173052817E0
:102A1000390719F484E695E1C4C10E947718009142
:102A20005B0C10915C0CD8018C918D3079F090E0AA
:102A30000E941E3F8536910561F4F801818190E086
:102A40000E941E3F8536910509F0A5C10E941D1404
:102A5000AAC18636910509F09EC1E8012196D801E8
:102A600011968C9190E00E941E3F8C36910509F0E2
:102A700092C12196D0935C0CC0935B0C0E9406100F
:102A80006C01BFEF8F3F9B0709F48DC1FC01EE0F76
:102A9000FF1FEE0FFF1FE050FF4F80819181A0E0EC
:102AA000B0E0EE24F82E092F1A2F2CE030E040E0A1
:102AB00050E0E20EF31E041F151F0BBFF7018791B4
:102AC000969124EF3FEF4FEF5FEFE20EF31E041FEE
:102AD000151F8F5F9F4FE1F08BE396E10E94B10DD0
:102AE000B601882777FD8095982F0E947F2189E283
:102AF00096E10E94B10D8BE493E00E94EC0D809171
:102B00004B0390E00E941E3F8937910509F04BC1AD
:102B100020917205309173056091560C7091570C9D
:102B2000922F961B40914E0F50914F0FE091BF0591
:102B3000F091C005A42FAE1B892F8A0F865E80936B
:102B40005F0C8FEF80937F031092730310927403D6
:102B500090937503261B370B3093760310927703FF
:102B600010927803A09379034E1B5F0B50937A0366
:102B700010927B0310927C038091B7059091B80569
:102B80002CEE3CE0482F421B40937D038C5E9C4022
:102B9000892F990F990B80937E03C801B70147E6EF
:102BA00053E00E9400FEF601EE0FFF1FEE0FFF1F25
:102BB000EE5FFE4F808191817C0100E010E0C0E07B
:102BC000D0E040E050E01EC0FA01E959FC4FDE01C0
:102BD000AA59B94F8C9180834F5F5F4F81E040309D
:102BE000580779F4902F8F2D7E2D662747E653E006
:102BF0000E9400FE0894E11CF11C011D111D40E023
:102C000050E0219680917205909173052091560CA9
:102C10003091570C821B930BC817D907A8F2452B8C
:102C200041F0902F8F2D7E2D662747E653E00E94BE
:102C300000FE0894E11CF11C011D111DC0E0D0E054
:102C400040E050E01EC0FA01E959FC4FDE01A458F3
:102C5000B14F8C9180834F5F5F4F91E040305907B7
:102C600079F4902F8F2D7E2D662747E653E00E9442
:102C700000FE0894E11CF11C011D111D40E050E014
:102C8000219680914E0F90914F0F2091BF0530916A
:102C9000C005821B930BC817D907A8F2452B41F03A
:102CA000902F8F2D7E2D662747E653E00E9400FE71
:102CB0000894E11CF11C011D111DC0E0D0E020E0D2
:102CC00030E01EC0F901E959FC4FDE01A451B34FB9
:102CD0008C9180832F5F3F4FA1E020303A0779F439
:102CE000902F8F2D7E2D662747E653E00E9400FE31
:102CF0000894E11CF11C011D111D20E030E021961B
:102D00008091B7059091B8058C5E9C40C817D90793
:102D1000C8F2232B41F0902F8F2D7E2D662747E69A
:102D200053E00E9400FE82E296E10E94B10D6091A4
:102D30007205709173052091560C3091570C621BEF
:102D4000730B882777FD8095982F0E947F218EE056
:102D500096E10E94B10D60914E0F70914F0F20913E
:102D6000BF053091C005621B730B882777FD8095E6
:102D7000982F0E947F2183EF95E10E94B10DB6014B
:102D8000882777FD8095982F0E947F215D9BFECF3D
:102D90008EE28CB908C08DE295E10E94B10D80E110
:102DA00095E10E94B10DDF91CF911F910F91FF909E
:102DB000EF90DF90CF900895EF92FF920F931F93C3
:102DC0009C018F3F910541F488E190E06FEF0E94F4
:102DD000FB138EEF96E15AC08535910591F48CE096
:102DE00090E00E94B6118F5F9F4F19F482EE96E13A
:102DF0004DC088E190E065E50E94FB138AEB96E107
:102E000045C08A35910511F460E00AC08B35910503
:102E100011F461E005C08C35910509F039C062E01C
:102E2000E62FF0E0EE0FFF1FEE0FFF1FE050FF4F09
:102E300080819181A0E0B0E0BA2FA92F982F882738
:102E40000C96A11DB11DABBFFC0187919691E62E9A
:102E5000FF2400E010E08F5F9F4F49F488E996E17E
:102E60000E94B10DC801B7010E947F2111C088E105
:102E700090E0622F0E94FB1381E896E10E94B10D61
:102E8000C801B7010E947F218AE696E10E94B10D38
:102E90001F910F91FF90EF900895DF92EF92FF92B4
:102EA0000F931F937B018C01D42ECB01652F0E94C1
:102EB000583F0894E11CF11CC7016D2D0E94583F3A
:102EC0001F910F91FF90EF90DF900895AF92BF9206
:102ED000CF92DF92EF92FF920F931F937B018C01B1
:102EE00059016A019A0144275527A9010E944D17EB
:102EF00082E090E0A0E0B0E0E80EF91E0A1F1B1F80
:102F0000C801B701A5010E944D171F910F91FF90B5
:102F1000EF90DF90CF90BF90AF900895DC01CB0190
:102F2000642F0E94583F08956F927F928F929F92D4
:102F3000BF92CF92DF92EF92FF920F931F93DF9396
:102F4000CF93CDB7DEB72F970FB6F894DEBF0FBE85
:102F5000CDBF4C01BB2413E1612E712C6E0108948E
:102F6000C11CD11C8B2D90E0869D7001879DF00CBB
:102F7000969DF00C11248701085A1C4EC8010E942E
:102F8000353F892BF9F0C601B8010E942E3FC601DA
:102F90000E946B19892BA1F0F701E959FC4E85912C
:102FA0009591A591B491F40180839183A283B38319
:102FB000F60101900020E9F73197EC19FD0904C0F2
:102FC000B394D0CFE0E0F0E0CF012F960FB6F894A5
:102FD000DEBF0FBECDBFCF91DF911F910F91FF904C
:102FE000EF90DF90CF90BF909F908F907F906F90E9
:102FF00008950E94EC1A81E090E00895FC0111828E
:103000004083738362830895FC011182408373833C
:1030100062830895FC018181882331F46093460C1A
:103020000E94F92180E00895815081830280F3811C
:10303000E02DE80FF11D80810895DC0111969C912F
:1030400011978C91981729F44093460C0E94F9210E
:1030500008951296ED91FC911397E90FF11D60838D
:1030600011968C9111978F5F11968C930895FC01A6
:103070008181882349F46093460C0E94F92120E065
:1030800030E040E050E010C08150818390E0880F34
:10309000991F880F991F0280F381E02DE80FF91F17
:1030A0002081318142815381B901CA010895DC0137
:1030B00011963C9111978C91381729F42093460C66
:1030C0000E94F9210895832F90E0880F991F880F9F
:1030D000991F1296ED91FC911397E80FF91F408309
:1030E0005183628373833F5F11963C93089505C0BB
:1030F0003196F0935C0CE0935B0CE0915B0CF091EB
:103100005C0C80818032A1F30895E0915B0CF0911A
:103110005C0C808190E0C0970A97E8F019C0CA0162
:10312000B3E0880F991FBA95E1F7440F551F480F78
:10313000591F460F571F3196F0935C0CE0935B0CC0
:103140004217530710F09A010AC081E08093460CA1
:1031500040E050E010C040E050E020E030E0E0917E
:103160005B0CF0915C0C8081682F70E060537040C4
:103170006A307105A0F2CA010895E091520CF091F5
:10318000530C81939193F093530CE093520C089558
:10319000E091520CF091530C91838083128233960C
:1031A000F093530CE093520C089590E006C03196D2
:1031B000F0935C0CE0935B0C9F5FE0915B0CF091F3
:1031C0005C0C8081803299F39923C1F0A091520C5C
:1031D000B091530C923058F0FD018FE78193119616
:1031E0009C933196F093530CE093520C0895FD019B
:1031F0008EE78193F093530CE093520C0895E09185
:103200005B0CF0915C0C8081089580915B0C909137
:103210005C0C019690935C0C80935B0C0895E0919C
:10322000520CF091530C6193719381939193F093AD
:10323000530CE093520C0895282FE091520CF0911A
:10324000530C809154069091550680589F4FE81773
:10325000F90721F484E18093460C0895208380913E
:10326000520C9091530C01969093530C8093520CF6
:103270000895AF92BF92CF92DF92FF920F931F9368
:10328000CF93DF935C016B01C0E0D0E013C0F50188
:10329000EC0FFD1F808190E00E94263F8C018F2D56
:1032A00090E00E94263F0817190719F0C0E0D0E00F
:1032B00007C02196F601EC0FFD1FF080FF2039F7C3
:1032C000CE01DF91CF911F910F91FF90DF90CF90B2
:1032D000BF90AF9008950F931F93182F092F8091DF
:1032E0005B0C90915C0C612F702F0E943919892B17
:1032F00019F4A0E0B0E013C0E12FF02FDF010D9032
:103300000020E9F71197AE1BBF0B80915B0C9091E9
:103310005C0C8A0F9B1F90935C0C80935B0CCD011F
:103320001F910F91089515C11092B9050E94D518EB
:103330008CE091E00E946B19892B19F00E94261CE9
:10334000F2C081E191E00E946B19892B19F00E9473
:10335000191EE9C085E191E00E946B19892B19F0D3
:103360000E940823E0C08AE191E00E946B19892B3A
:1033700019F00E945E21D7C082E291E00E946B1991
:10338000892B19F00E94461ECEC088E291E00E946F
:103390006B19892B19F00E94421EC5C08DE291E085
:1033A0000E946B19892B19F00E946924BCC080E32C
:1033B00091E00E946B19892B19F00E94BE1BB3C0CB
:1033C00087E391E00E946B19892B19F00E94D323A7
:1033D000AAC08AE391E00E946B19892B19F00E9420
:1033E0002923A1C080E491E00E946B19892B19F078
:1033F0000E94BB2298C086E491E00E946B19892B41
:1034000019F00E9463238FC08AE491E00E946B1937
:10341000892B19F00E94152386C08FE491E00E9449
:103420006B19892B19F00E94C91B7DC084E591E0BE
:103430000E946B19892B19F00E94692174C08AE5DA
:1034400091E00E946B19892B19F00E94D41B6BC06C
:103450008EE591E00E946B19892B19F00E942E1CB9
:1034600062C082E691E00E946B19892B19F00E94DC
:10347000F62259C086E691E00E946B19892B19F05B
:103480000E94DF1B50C08BE691E00E946B19892BD4
:1034900019F00E94EA1B47C081E791E00E946B1976
:1034A000892B19F00E9457223EC087E791E00E94C5
:1034B0006B19892B19F00E94D82535C08DE791E052
:1034C0000E946B19892B19F00E94D4252CC083E827
:1034D00091E00E946B19892B19F00E94DC2523C012
:1034E00087E891E00E946B19892B19F00E94BF2296
:1034F0001AC08EE891E00E946B19892B19F00E9486
:10350000B72211C080E991E00E946B19892B19F054
:103510000E942A1C08C082E991E00E946B19892B45
:1035200091F50E94151E8091460C882361F50E943A
:10353000D518E0915B0CF0915C0CE081EA3319F452
:103540000E94AA1B06C0ED3021F082E08093460C59
:103550000895E0915B0CF0915C0C80818D3009F056
:10356000E3CEE091520CF091530C8DE78083809173
:10357000BE05882341F42091520C88E59FE0281B6A
:103580002F5F20935A0F08951F93182F90E00E94E9
:103590000C3F892B39F420E030E0812F90E0C09778
:1035A0000A9710F421E030E0C9011F9108950F93AC
:1035B0001F9300E61CE0C8010E94EC0DF801019089
:1035C0000020E9F731978DE0808310935C0C009325
:1035D0005B0C1F910F910895DF92EF92FF920F9372
:1035E0001F93DF93CF9300D0CDB7DEB70E943E1379
:1035F0000E94632D0E944E2D87EB95E0BE016F5F08
:103600007F4F0E944A0D8091B7059091B80529819E
:103610003A81820F931F90934B0F80934A0F0E9421
:10362000C912892B11F00E942C290E94720D0E9450
:10363000720D0E94BF0D8DE797E10E94B10D8DE3E1
:1036400097E10E94B10D81E08093BE0518E5E12E5F
:103650001FE0F12EDD24D3948091BE05882321F054
:1036600081E997E10E94B10D1092BE051092460CBF
:1036700010924E060E94720D8EE30E94D00D0E94A1
:10368000D71A05C03196F0935C0CE0935B0CE09187
:103690005B0CF0915C0C80818032A1F380EE9CE0A9
:1036A00069E975E04EE10E94041884EE9CE06BE746
:1036B00074E04CE30E94FE170E94302C892B61F6C7
:1036C00000914E0F10914F0FF092530CE092520C5C
:1036D000109298050E9485189C010097D1F0E09106
:1036E0005B0CF0915C0C80818D3021F4C9010E944B
:1036F000AA2D24C01092BE05E091520CF091530CFB
:103700003183208312823396F093530CE093520C52
:1037100002C0D092BE058091460C882379F40E94A5
:1037200093198091460C882349F48091BE05882323
:1037300019F00E94E72602C00E948E2E8091460C4E
:10374000882309F489CF0E94F92110934F0F009329
:103750004E0F82CFE091520CF091530C8AE7819387
:10376000F093530CE093520C80915B0C90915C0CA5
:10377000019690935C0C80935B0C0895E091520C41
:10378000F091530C84E18193F093530CE093520C2D
:103790000895E091520CF091530C87E18193F093DE
:1037A000530CE093520C0895E091520CF091530C9D
:1037B00088E18193F093530CE093520C0895E091CB
:1037C000520CF091530C86E08193F093530CE093EC
:1037D000520C0895E091520CF091530C87E08193C4
:1037E000F093530CE093520C0895A091520CB091B9
:1037F000530CFD01819311961C9211973196F09311
:10380000530CE093520C22E0E0915B0CF0915C0CC5
:103810008191F0935C0CE0935B0CE091520CF09181
:10382000530C8193F093530CE093520C8D3011F0B4
:103830002F5FEACF80915B0C90915C0C0197909385
:103840005C0C80935B0C11962C9308958CE00E9485
:10385000F51B089584E40E94F51B08958AE00E94F8
:10386000F51B089587E991E00E946B19892B11F0EF
:1038700082E308958AE991E00E946B19892B11F087
:1038800083E308958DE991E00E946B19892B11F073
:1038900085E3089580EA91E00E946B19892B11F06D
:1038A00080E3089582EA91E00E946B19892B11F060
:1038B00081E3089584EA91E00E946B19892B11F449
:1038C00080E0089584E3089586EA91E00E946B19F0
:1038D000892B11F080E208958AEA91E00E946B1929
:1038E000892B11F081E208958DEA91E00E946B1915
:1038F000892B11F480E0089582E2089581EB91E034
:103900000E946B19892B11F080E4089583EB91E0FC
:103910000E946B19892B11F081E4089585EB91E0E9
:103920000E946B19892B11F080E5089587EB91E0D7
:103930000E946B19892B11F081E5089589EB91E0C4
:103940000E946B19892B11F082E508958DEB91E0AF
:103950000E946B19892B11F480E0089580E6089588
:103960009F92AF92BF92CF92DF92EF92FF920F930E
:103970001F93182F00E061E7962E50E7B52E43E71E
:10398000A42E34E7D32E22E7C22E90E1E92E81E166
:10399000F82E0E94D51883EB91E00E946B19892BB9
:1039A00031F0E091520CF091530CC1922FC08FEB8B
:1039B00091E00E946B19892B31F0E091520CF0914B
:1039C000530CD19223C083EC91E00E946B19892B98
:1039D00031F0E091520CF091530CA19217C087EC9A
:1039E00091E00E946B19892B31F0E091520CF0911B
:1039F000530CB1920BC089EC91E00E946B19892B9A
:103A000049F0E091520CF091530C9192F093530CC9
:103A1000E093520C0E94D518E0915B0CF0915C0C85
:103A200080818832B9F5E091520CF091530CE1920B
:103A3000F093530CE093520C80915B0C90915C0CD2
:103A4000019690935C0C80935B0C812F0E94B01CBC
:103A50008091460C882309F077C0E0915B0CF091CF
:103A60005C0C8081893211F084E060C0E091520CDE
:103A7000F091530CF192F093530CE093520C80911F
:103A80005B0C90915C0C019690935C0C80935B0CAA
:103A900011E01EC00E94B61F982F882369F40E946F
:103AA000E025982F882341F40E94B70F982F882390
:103AB00019F40E949420982F8091460C882309F0D5
:103AC00043C0112321F0911711F085E02FC0192F69
:103AD0000E94D518E0915B0CF0915C0CE081ED3018
:103AE00099F1EA3389F1EC3279F1EB3369F1E9329A
:103AF00059F11130C1F40E947E1C8823D9F40E9430
:103B0000641C8823B9F48091B905882339F0002317
:103B1000D9F40E94321C882361F407C08091F90F08
:103B2000882319F011C083E101C086E08093460C20
:103B30000BC001E0E091520CF091530C8193F09393
:103B4000530CE093520C25CF1F910F91FF90EF90F3
:103B5000DF90CF90BF90AF909F9008951F930E94E9
:103B6000B70F182F882329F40E949420182F882338
:103B700011F18091460C8823F1F40E94D518E09150
:103B80005B0CF0915C0C8191F0935C0CE0935B0C0E
:103B90008D3321F083E08093460C0DC0E091520CF0
:103BA000F091530C89E78193F093530CE093520CFE
:103BB000812F0E94B01C1F910895E091520CF0914A
:103BC000530C8193F093530CE093520C0E94D51840
:103BD00083EC91E00E946B19892B31F0E091520C3B
:103BE000F091530C83E717C08FEB91E00E946B19A3
:103BF000892B31F0E091520CF091530C84E70BC00B
:103C000087EC91E00E946B19892B51F0E091520CE6
:103C1000F091530C80E78193F093530CE093520C96
:103C20000E94D5180E94AE1D089582E00E94DD1DFD
:103C3000089581E00E94DD1D0895E091520CF091FD
:103C4000530C8193F093530CE093520C0E94D518BF
:103C5000E091520CF091530C88EA8193F093530C4D
:103C6000E093520C0E9485189C01009719F482E1A0
:103C70008093460C8091460C882319F4C9010E9458
:103C8000BD18089582E10E941D1E08958FE00E94D4
:103C90001D1E0895E0915B0CF0915C0C80818832D0
:103CA00019F424E930E002C020E030E0C9010895B1
:103CB000282FDB0140914E0F50914F0FFA01819355
:103CC000F0934F0FE0934E0F90E08C91E0914E0FE8
:103CD000F0914F0F8193F0934F0FE0934E0F8C9123
:103CE000811111969F5F9E3081F7243851F024395D
:103CF00041F0223811F494E005C0213811F088E039
:103D00001BC095E081E020914E0F30914F0FF901DB
:103D10001192F0934F0FE0934E0F8F5F981798F723
:103D200030934F0F20934E0F80914B0C90914C0C81
:103D30008217930730F489E08093460CEFEFFFEF92
:103D400007C08091BF059091C005FA01E81BF90BEF
:103D5000CF0108950F931F93CF93DF93E0915B0CF6
:103D6000F0915C0C808190E0C0970A9728F420E0E5
:103D700030E040E050E025C082E016C0CA01B90141
:103D80002AE030E040E050E00E948E3E9B01AC0112
:103D9000CE01AA2797FDA095BA2F280F391F4A1FD9
:103DA0005B1F57FF08C08AE08093460C20E030E09C
:103DB00040E050E012C00F5F1F4F10935C0C009367
:103DC0005B0C00915B0C10915C0CF8018081C82F9A
:103DD000D0E0E097CA30D10588F2B901CA01DF917D
:103DE000CF911F910F910895CF93DF93C091520C03
:103DF000D091530CDE0182EA8D93CD010196909310
:103E0000530C8093520CE0915B0CF0915C0C21916F
:103E100011962C9301969093530C8093520CF0932F
:103E20005C0CE0935B0C22E018C08D3019F4809399
:103E3000460C2DC0E091520CF091530C8193F093FD
:103E4000530CE093520C80915B0C90915C0C0196AA
:103E500090935C0C80935B0C2F5FE0915B0CF09176
:103E60005C0C8081823209F7E091520CF091530C86
:103E70008193F093530CE093520C80915B0C9091E2
:103E80005C0C019690935C0C80935B0C2983DF9112
:103E9000CF91089590E00E94133F0895BF92CF9272
:103EA000DF92EF92FF920F931F93CF93DF93E091F6
:103EB0005B0CF0915C0C808190E00E94133F892B99
:103EC00029F0EE24FF248701BB2433C08BE023C0FC
:103ED0009E0120533040D801C70144E0880F991F4C
:103EE000AA1FBB1F4A95D1F72A30310530F479015A
:103EF0000027F7FC0095102F06C0E7977E010027EA
:103F0000F7FC0095102FE80EF91E0A1F1B1F89E011
:103F1000B81639F48CE08093460CEE24FF24870118
:103F200019C0B3940894C11CD11CD0925C0CC092EF
:103F30005B0CC0905B0CD0905C0CF601808190E033
:103F40000E94263FC82FD0E0CE010E94133F892B4C
:103F500009F0BECFB701C801DF91CF911F910F913A
:103F6000FF90EF90DF90CF90BF9008950F931F9335
:103F7000DF93CF9300D000D0CDB7DEB700915B0CBC
:103F800010915C0CF8018081823229F40E94F41EA9
:103F900022E030E04FC0843259F40F5F1F4F10937E
:103FA0005C0C00935B0C015010400E944E1F0EC031
:103FB00090E00E940C3F892B39F0CE0101960E94BF
:103FC0009417882339F434C00E94AA1E69837A8327
:103FD0008B839C838091460C882351F5E091520C91
:103FE000F091530C84EA8193F093530CE093520CBC
:103FF00069817A818B819C810E940F1980915B0C71
:10400000801B03C0F80181918F01E091520CF09167
:10401000530C8193F093530CE093520C80915B0C02
:1040200090915C0C0817190768F321E030E002C09A
:1040300020E030E0C9010F900F900F900F90CF91CA
:10404000DF911F910F910895CF93DF93EC01E881E9
:10405000F9818081843981F47396F983E8837397B9
:1040600087859089009701F1DC012D913D91220F08
:10407000331F220F331F10C0843841F4DF011F9615
:104080007396F983E88324E030E006C088E08093EB
:10409000460C0E94F92108C080E090E002C01D9209
:1040A000019682179307D8F3DF91CF910895EF928D
:1040B000FF920F931F93CF93DF93E82E8B01FB01A9
:1040C00001900020E9F73197FE2EF61AC091BF0546
:1040D000D091C0051CC08E1581F4BE016F5F7F4F6B
:1040E000C8010E943919F81641F48091BF059091DA
:1040F000C005BE01681B790B0FC08881843831F080
:10410000843921F088E08093460C04C0639688814E
:10411000882309F76FEF7FEFCB01DF91CF911F91DC
:104120000F91FF90EF9008951F93CF93DF93E7E6F1
:10413000F4E0119284E0E637F807D9F7C0915B0C00
:10414000D0915C0C1881812F90E00E940C3F892B4C
:1041500041F0109367042196D0935C0CC0935B0CE4
:1041600003C087E08093460CC8E6D4E0E0915B0C86
:10417000F0915C0C80810E94C41A892B71F0E0914F
:104180005B0CF0915C0C81918993F0935C0CE09353
:104190005B0C84E0C537D80749F7E0915B0CF091E0
:1041A0005C0C8081883219F484E990E002C080E0E0
:1041B00090E080937604882321F484E88093760449
:1041C00005C03196F0935C0CE0935B0C8091460C3B
:1041D000882309F051C08091760467E674E00E945C
:1041E00057209C018091460C882309F045C08FEF31
:1041F0002F3F3807C1F490917604943931F48091BF
:104200009805882311F488E135C0892F67E674E0AA
:104210000E94581E9C018FEF2F3F380769F1809153
:10422000460C882349F580917604E091520CF09178
:10423000530C8193F093530CE093520CC9010E94EC
:10424000BD1880917604843949F5E091520CF091C3
:10425000530C80E18193F093530CE093520C81E076
:104260000E94B01CE0915B0CF0915C0C8081893263
:1042700031F08EE08093460C20E030E01AC0319699
:10428000F0935C0CE0935B0CE091520CF091530CBA
:1042900081E18193F093530CE093520C809176046A
:1042A000843829F0843919F022E030E002C021E09E
:1042B00030E0C901DF91CF911F910895E091520C38
:1042C000F091530C8EE08193F093530CE093520CD9
:1042D0000895E091520CF091530C8AE18193F09390
:1042E000530CE093520C0895E091520CF091530C52
:1042F0008CE08193F093530CE093520C08958F92CD
:104300009F92AF92BF92CF92DF92EF92FF920F9364
:104310001F93DF93CF93CDB7DEB764970FB6F894B2
:10432000DEBF0FBECDBF7B018C011C8A97FF11C081
:104330008DE20E94D00DAA24BB246501AE18BF08EF
:10434000C00AD10A82E1F82E4E010894811C911C0A
:1043500026C0611571058105910519F05B016C019D
:10436000F1CF80E30E94D00D28C0080D191DC601B1
:10437000B5012AE030E040E050E00E94CD3E605DB3
:10438000F8016083FA94C601B5012AE030E040E00C
:1043900050E00E94CD3EC901DA015C016D010F2D94
:1043A00010E0A114B104C104D104F9F60F5F1F4F4E
:1043B000C401800F911F0E94C40D64960FB6F8943B
:1043C000DEBF0FBECDBFCF91DF911F910F91FF9048
:1043D000EF90DF90CF90BF90AF909F908F90089517
:1043E00098E2899FC00111248C599F4F0E94B10D02
:1043F0000895CF93DF9380914E068823D1F085EB0B
:1044000097E10E94B10D6091460C70E080E090E071
:104410000E947F218BEA97E10E94B10D60915D0CB3
:1044200070915E0C80E090E00E947F2188EA97E125
:1044300032C00E94720D0E94720DC0E6DCE002C024
:104440000E94D00D89918D30D9F70E94720D20E61F
:104450003CE004C08AE20E94D00D9E01E901219651
:1044600080915B0C90915C0C02972817390790F3B0
:1044700084EA97E10E94B10D0E94720D8CE997E1E8
:104480000E94B10D6091460C70E080E090E00E94C7
:104490007F2189E997E10E94B10D8091460C0E942D
:1044A000F02181E08093430CDF91CF9108958091BA
:1044B000B9058F5F8093B905E091520CF091530CD0
:1044C00089E18193F093530CE093520C80E00E94B9
:1044D000B01C08950F931F93E091520CF091530C70
:1044E0008193F093530CE093520C0E94D5180BE784
:1044F0001CE731C080E00E94B01C8091460C8823EC
:1045000099F50E94D518E0915B0CF0915C0CE0816C
:10451000EC3231F4E091520CF091530C108307C04F
:10452000EB3311F5E091520CF091530C0083809124
:104530005B0C90915C0C019690935C0C80935B0CEF
:104540008091520C9091530C01969093530C809350
:10455000520C0E94D518E0915B0CF0915C0CE0814C
:10456000ED3011F0EA3331F61F910F91089583E495
:104570000E946A22089583E00E946A220895E091D1
:10458000520CF091530C83E28193F093530CE0931F
:10459000520C0E94D5180E94942008951F931CE786
:1045A0000E94D5180E9494208091460C8823E1F443
:1045B0000E94D518E0915B0CF0915C0C80818C32EC
:1045C00099F4E091520CF091530C1193F093530C29
:1045D000E093520C80915B0C90915C0C019690934F
:1045E0005C0C80935B0CDCCF1F91089581E080937D
:1045F0009805E091520CF091530C89E08193F0936F
:10460000530CE093520C0E94CE221092980508950C
:10461000E091520CF091530C8DE08193F093530C88
:10462000E093520C0E94CE220895E091520CF0913A
:10463000530C85E08193F093530CE093520C0E944D
:10464000D5180E949420019719F082E08093460CBF
:104650000895E091520CF091530C86E18193F09310
:10466000530CE093520C0E94D518E0915B0CF09132
:104670005C0C8081823221F50E94F41E8091460CF0
:10468000882301F5E0915B0CF0915C0C80818C3209
:1046900021F082E08093460C0895E091520CF09155
:1046A000530C8CE78193F093530CE093520C809160
:1046B0005B0C90915C0C019690935C0C80935B0C6E
:1046C0000E94CE2208951F9381E08093F90FE0911C
:1046D000520CF091530C84E08193F093530CE093CF
:1046E000520C0E94D5180E949420182F0E94D518B1
:1046F000113059F4E0915B0CF0915C0C8191F093D6
:104700005C0CE0935B0C8D3311F083E02EC0E091E4
:10471000520CF091530C89E78193F093530CE09382
:10472000520C81E00E94B01C8091460C8823C9F590
:104730000E94D5188DEC91E00E946B19892BA1F095
:10474000E091520CF091530C87E38193F093530C5A
:10475000E093520C0E94D51881E00E94B01C809119
:10476000460C8823F1F404C081E18093460C19C003
:104770000E94D51880ED91E00E946B19892B79F089
:10478000E091520CF091530C8AE38193F093530C17
:10479000E093520C0E94D51881E00E94B01C109248
:1047A000F90F1F910895E091520CF091530C85E19F
:1047B0008193F093530CE093520C0E94D518809192
:1047C000B9058F5F8093B90581E00E94B01C80918C
:1047D000460C882309F07CC00E94D51885ED91E035
:1047E0000E946B19892BB9F1E091520CF091530C96
:1047F00088E38193F093530CE093520C0E94D518F8
:10480000E0915B0CF0915C0C808190E0C0970A977E
:10481000D8F4E091520CF091530C88EA8193F09314
:10482000530CE093520C0E9485189C01009719F4D8
:1048300082E18093460C8091460C882309F048C0A1
:10484000C9010E94BD180BC00E9493198091460CAB
:10485000882329F0089580E18093460C08950E94F2
:10486000D5188AED91E00E946B19892B89F1E091AE
:10487000520CF091530C89E38193F093530CE09325
:10488000520C0E94D518E0915B0CF0915C0C808179
:1048900090E0C0970A97D0F4E091520CF091530C3D
:1048A00088EA8193F093530CE093520C0E94851890
:1048B0009C01009719F482E18093460C8091460C8C
:1048C000882331F4C9010E94BD1808950E949319EC
:1048D0000895FF920F931F93E091520CF091530CA7
:1048E00083E18193F093530CE093520C0E94D5180E
:1048F00081E00E94B01C8091460C882309F056C0CC
:104900000E94D5188FED91E00E946B19892B19F048
:104910000E94421E0CC084EE91E00E946B19892B0C
:1049200019F00E94461E03C08FE08093460C8091D0
:10493000460C8823D9F50E94D5189CE7F92E08EA81
:1049400012E12DC0E091520CF091530CF192F093D2
:10495000530CE093520C80915B0C90915C0C01968F
:1049600090935C0C80935B0C0E94D518E091520CE4
:10497000F091530C0193F093530CE093520C0E946E
:1049800085189C01009711F41093460C8091460CF9
:10499000882361F4C9010E94C8180E94D518E091CB
:1049A0005B0CF0915C0C80818C3261F21F910F9155
:1049B000FF900895DF92EF92FF920F931F93CF9392
:1049C000DF938B017A01C091520CD091530CDE0120
:1049D0008D93B093530CA093520CE0915B0CF0912B
:1049E0005C0C8081883239F580E189831196B0931F
:1049F000530CA093520C80915B0C90915C0C01962F
:104A000090935C0C80935B0C8CE7D82EF70181911E
:104A10007F010E94B01C8091460C8823D9F501507B
:104A20001040E0915B0CF0915C0C01151105C1F098
:104A300080818C3211F082E017C0E091520CF0912D
:104A4000530CD192F093530CE093520C80915B0C79
:104A500090915C0C019690935C0C80935B0CD6CF8C
:104A60008081893221F08EE08093460C13C0E09162
:104A7000520CF091530C81E18193F093530CE0932D
:104A8000520C80915B0C90915C0C019690935C0CA5
:104A900080935B0CDF91CF911F910F91FF90EF906E
:104AA000DF900895DF93CF930F92CDB7DEB791E0FB
:104AB000998361E070E0AE014F5F5F4F0E94DA249E
:104AC00081E00F90CF91DF91089583E10E945225FC
:104AD000089582E10E94522508958AE00E9452259D
:104AE000089580E10E94522508958FE00E9452258A
:104AF000089589E00E94522508958EE00E94522573
:104B000008958DE00E94522508958BE00E94522561
:104B100008958CE00E945225089583E00E9452255A
:104B200090E0089581E10E94522508958BE00E9453
:104B30005225089587E00E94522590E0089586E06E
:104B40000E94522590E0089585E00E94522590E051
:104B5000089584E00E94522590E0089582E00E942A
:104B6000522590E008950E9452250E94D518E091A8
:104B70005B0CF0915C0C8191F0935C0CE0935B0C0E
:104B80008D3321F083E08093460C0895E091520C20
:104B9000F091530C89E78193F093530CE093520CFE
:104BA00081E00E94B01C08958DE10E94B325089514
:104BB0008CE10E94B32508958BE10E94B3250895EE
:104BC000CF93DF93C091520CD091530C86E388832E
:104BD0008091520C9091530C01969093530C8093BA
:104BE000520C8AEE91E00E946B19892B19F00E94F9
:104BF000AE2595C08FEE91E00E946B19892B19F0BC
:104C00000E94A9258CC083EF91E00E946B19892B2B
:104C100019F00E948D2583C088EF91E00E946B19E6
:104C2000892B19F00E94A4257AC08CEF91E00E9494
:104C30006B19892B19F00E949F2571C080E092E0CA
:104C40000E946B19892B19F00E949A2568C084E094
:104C500092E00E946B19892B19F00E947D255FC09C
:104C600089E092E00E946B19892B19F00E9481253E
:104C700056C08EE092E00E946B19892B19F00E94B9
:104C800085254DC082E192E00E946B19892B19F0B5
:104C90000E94752544C089E192E00E946B19892B1E
:104CA00019F00E9471253BC080E292E00E946B19CE
:104CB000892B19F00E94792532C085E292E00E948A
:104CC0006B19892B19F00E94922529C08AE292E083
:104CD0000E946B19892B19F00E94692520C080E37E
:104CE00092E00E946B19892B19F00E94652517C06C
:104CF00086E392E00E946B19892B19F00E946D25C2
:104D00000EC08AE392E00E946B19892B19F00E9471
:104D1000892505C0D093530CC093520C80E0DF91DD
:104D2000CF9108951F93CF93DF93DB01EC018A812C
:104D30006AE00E94AD3E805DFD0181938A810E9400
:104D4000AD3E905D11969C93DF0111961AE311839D
:104D5000AD014F5F5F4F89810E94AD3E805D11962E
:104D60008C93FA01319689810E94AD3E905DDA0103
:104D700011969C93DF0111961183FD013196888174
:104D80000E94AD3E805D11968C9388810E94AD3E5D
:104D9000905D91831282DF91CF911F9108950895C4
:104DA0000895E091520CF091530C80818E3719F0E8
:104DB0008F3761F406C03196F093530CE093520C98
:104DC00008953296F093530CE093520C089588E5C1
:104DD0009FE09093530C8093520C0E94D1261DC0EB
:104DE0000E94D126E091520CF091530C8191F093E6
:104DF000530CE093520C90E001979C01220F331F5B
:104E0000280F391F220F331F220F331F2452354F13
:104E1000F90185919491FC010995E091520CF09172
:104E2000530C80818D3721F08091460C8823C1F28C
:104E300008958AE08093540F8091510C882371F07B
:104E40001092510C89E38093460C809176059091E5
:104E500077059093570F8093560F81E008950F9335
:104E60001F93DF93CF9300D0CDB7DEB70E944E2DB6
:104E70008091BF059091C0059A8389838E010F5F51
:104E80001F4F03C0C8010E942420E981FA8180815C
:104E90008823C1F70F900F90CF91DF911F910F9151
:104EA00008950E942F271092510C1092550F8AE0FE
:104EB0008093540F1092430C10925F0610925E067E
:104EC0000895DF93CF93CDB7DEB764970FB6F8940C
:104ED000DEBF0FBECDBF2091560C3091570C809194
:104EE0007205909173052817390791F087EE97E1C5
:104EF0000E94B10DCE0101960E94EC0D8981893787
:104F000011F0893549F40E94632D85ED97E102C0C7
:104F10008DEB97E10E94B10D64960FB6F894DEBF59
:104F20000FBECDBFCF91DF91089507C03196F093AA
:104F30007804E09377040E94D00DE0917704F0911B
:104F4000780480818D3791F708950F931F93CF9345
:104F5000DF93A0917704B0917804FD012191F09343
:104F60007804E09377042633F1F1273330F42A30C4
:104F700021F12C3009F04DC026C02E37D1F02F374B
:104F800021F0243409F045C01BC011968C91319654
:104F9000F0937804E0937704C0E0D0E0082F10E0AD
:104FA00004C080E20E94D00D2196C017D107CCF337
:104FB00040C080E20E94D00D3CC084E498E105C06E
:104FC00082E498E102C08DE398E10E94B10D8091E6
:104FD00077049091780401969093780480937704F5
:104FE0000E94952726C011962C913196F093780453
:104FF000E093770430E021503040C901880F991FB9
:10500000820F931F880F991F880F991F8251964F07
:105010000EC030E021503040C901880F991F820F27
:10502000931F880F991F880F991F8252954F0E94D6
:10503000B10DDF91CF911F910F9108951F9390E0D3
:105040000196E0917704F0917804E80FF91FF0934E
:105050007804E09377041191F0937804E093770457
:105060000CC0E0917704F09178048191F09378047A
:10507000E09377040E94D00D1150112391F71F91F6
:10508000089580E00E941E28089584E00E941E2852
:10509000089584E00E941E2808950F931F93CF93D4
:1050A000DF93E0917704F0917804818192813396C7
:1050B000F0937804E0937704C091BF05D091C005C8
:1050C000C80FD91F8E01025F1F4F8981882311F0FD
:1050D0000E94D00D2196C017D107B9F7DF91CF916B
:1050E0001F910F9108950E944D280895E091520C50
:1050F000F091530C82819F01280F311D3093770569
:10510000209376058191919190935E0C80935D0C34
:10511000F093530CE093520C80916B05882389F037
:105120008BE50E94D00D60915D0C70915E0C80E06B
:1051300090E00E947F218DE50E94D00D80E20E94C8
:10514000D00D0895E0917704F09178046181728127
:105150003396F0937804E0937704882777FD809561
:10516000982F0E947F2108955CC00E94762880912C
:10517000520C9091530C01969093530C8093520CC7
:105180003AC00E94D126E091520CF091530C8191CB
:10519000F093530CE093520C8F3041F40E940D3782
:1051A0008091460C882309F041C082E190E001978C
:1051B0009C01220F331F280F391F220F331F220F8C
:1051C000331F2452354FF90185919491FC010995C3
:1051D0008091460C882351F58091540F882319F053
:1051E00081508093540F8091540F882321F40E94A2
:1051F00019278823D9F4E091520CF091530C808147
:105200008D3709F0BECF9F012F5F3F4F8091720510
:10521000909173052817390749F03093530C209368
:10522000520C8091460C882309F49FCF08958091F9
:10523000430C882359F48091560F9091570F909307
:10524000530C8093520C0E94B428089585E28093F9
:10525000460C0E94F92108950E94720D0E94512768
:1052600081E080934E062091560C3091570C80912E
:105270007205909173052817390729F48EE198E19A
:105280000E94B10D08953093530C2093520C30932B
:105290007705209376050E94B4288091460C8823D8
:1052A00011F00E94F9210E94720D08950F931F932F
:1052B000DF93CF93CDB7DEB72F970FB6F894DEBF4D
:1052C0000FBECDBFE0917704F09178048181928187
:1052D0003396F0937804E09377048E010F5F1F4FAD
:1052E000B8010E94A50FC8010E94C40D2F960FB6E9
:1052F000F894DEBF0FBECDBFCF91DF911F910F910C
:105300000895E0917704F0917804E081E93870F431
:10531000E13821F0E238D9F1E43819F40E944D283F
:105320000895E33869F50E9456290895E93A60F531
:10533000E13A19F40E9449280895E23A19F40E94CA
:1053400041280895E83A19F40E94A2280895E43A01
:1053500019F40E9445280895E43991F40E944D28DB
:1053600007C0E7FF03C00E94812902C00E94A52751
:10537000E0917704F0917804E081ED3791F708959A
:1053800088E08093460C089588E08093460C089549
:105390006F927F928F929F92AF92BF92CF92DF9245
:1053A000EF92FF920F931F93DF93CF93CDB7DEB7AA
:1053B000CF58D0400FB6F894DEBF0FBECDBF0E94CD
:1053C0007718E0915B0CF0915C0C1081812F90E0DC
:1053D0000E940C3F892B09F43EC180E492E00E94B8
:1053E0006B19892B09F43EC00E94720D86E492E08D
:1053F0000E94C40DEE24FF248E010F5F1F4FC701D2
:1054000065E070E00E94B93E892B11F40E94720D94
:10541000C701B8010E94A50F8981882301F1F80115
:1054200001900020E9F73197E01BF10B3E9738F02F
:105430001F860EC0C80167E572E00E943E3FF8017A
:1054400001900020E9F73197E01BF10B3E9790F3B4
:10545000C8010E94C40D0894E11CF11CD0CF0E9429
:10546000720DF6C089E592E00E946B19892B09F450
:1054700071C00E94720D1091BF050091C0058EE5AC
:1054800092E00E94C40D812F902F6C017601089448
:10549000E11CF11CAA24BB2490E1892E912C54C05C
:1054A000C50183709070892B11F40E94720DF60172
:1054B00080818438D1F4C7010E94C40DF7010190A6
:1054C0000020E9F73197EE19FF0984010E1B1F0B2D
:1054D00006C087E592E00E94C40D015010400115FE
:1054E0001105B9F783E792E024C0843909F0B0C010
:1054F000C7010E94C40D88E792E00E94C40D8AE7AC
:1055000092E00E94C40DF70101900020E9F7319765
:10551000EE19FF0984010E1B1F0B06C087E592E000
:105520000E94C40D0150104001151105B9F78CE718
:1055300092E00E94C40D0894A11CB11C83E190E08C
:10554000C80ED91EE80EF91EF6018081882309F0E5
:10555000A7CF7EC08FE792E00E946B19892B09F4D8
:1055600073C0A0907704B0907804EE24FF248701E4
:1055700080E1882E912C8C0E9D1EB2E16B2E712C39
:105580006C0E7D1E8CE698E10E94B10DC801B7013A
:105590000E947F2189E698E10E94B10D8E2D0E9424
:1055A000C00EAB01BC014115510561057105A9F1A2
:1055B000C40120E830E00E94DA0EF401C080D180FE
:1055C0007092780460927704FFEFCF16FFEFDF064A
:1055D00019F48CE598E123C080E20E94D00DB60159
:1055E00080E090E00E947F21809177049091780480
:1055F0000196909378048093770407C0E7FF03C077
:105600000E94812902C00E94A527E0917704F091B1
:105610007804E081ED3791F704C088E498E10E94B6
:10562000B10D0E94720D0894E11CF11C011D111DA9
:1056300083E0E816F1040105110509F0A3CFB0924B
:105640007804A092770404C085E892E00E94C40D1B
:105650000E94720DACC0812F90E0C097E091560C73
:10566000F091570C20917205309173050A97A0F5BF
:10567000E217F30709F49BC00E9485189093650612
:10568000809364060E947718E0915B0CF0915C0CAB
:1056900080818D32C1F43196F0935C0CE0935B0C09
:1056A0000E947718E0915B0CF0915C0C808190E097
:1056B000C0970A9718F40E94851809C08091500F6E
:1056C0009091510F04C0809164069091650690936B
:1056D000500680934F0612C0E217F30709F467C023
:1056E0008091500F9091510F9093500680934F06E8
:1056F0008081918190936506809364062091640671
:105700003091650680914F0690915006821793075D
:1057100008F44DC0C9010E947F2D909378048093B6
:1057200077040E94720DE0917704F09178048091E3
:10573000720590917305E817F907C8F50191119169
:10574000F0937804E093770480914F06909150068F
:105750008017910760F180E20E94D00DB80180E0CF
:1057600090E00E947F2180917704909178040196C7
:10577000909378048093770407C0E7FF03C00E94EA
:10578000812902C00E94A527E0917704F091780456
:10579000E081ED3791F70E94720D8091770490912E
:1057A000780401969093780480937704BCCFC15716
:1057B000DF4F0FB6F894DEBF0FBECDBFCF91DF91A4
:1057C0001F910F91FF90EF90DF90CF90BF90AF901F
:1057D0009F908F907F906F900895DF92EF92FF924D
:1057E0000F931F937C018B01DC0113968C9113970F
:1057F0006AE00E94AD3E805DF801819313968C9122
:105800000E94AD3E905DD80111969C9320E2D22E6D
:10581000D182CF0102966BEC72E00E94493FF80101
:10582000D682D70115968C91159764E60E94AD3EFD
:10583000892F6AE00E94AD3E805D878315968C912A
:1058400064E60E94AD3E892F6AE00E94AD3E905D05
:10585000908711861F910F91FF90EF90DF90089530
:105860008FEC92E00E946B19892B19F00E94C829D5
:105870004AC084ED92E00E946B19892B19F00E94B6
:105880002C2941C088ED92E00E946B19892B19F0F8
:105890000E94612738C08CED92E00E946B19892B21
:1058A00019F00E9417292FC081EE92E00E946B1917
:1058B000892B19F00E942F2726C087EE92E00E94C4
:1058C0006B19892B19F00E948A2C1DC08CEE92E076
:1058D0000E946B19892B19F00E947D1214C081EF70
:1058E00092E00E946B19892B19F00E94F7140BC0EB
:1058F00086EF92E00E946B19892B19F420E030E0CA
:1059000004C00E94DB2C21E030E0C9010895089515
:10591000089508950E94720D84EC98E10E94B10DE3
:105920006091440C7091450C209172053091730583
:10593000621B730B882777FD8095982F0E947F212B
:1059400088EB98E10E94B10D0E94720D86EA98E101
:105950000E94B10D60914B0C70914C0C20914E0F38
:1059600030914F0F621B730B882777FD8095982F1E
:105970000E947F218AE998E10E94B10D0E94720D78
:105980008BE798E10E94B10D60914A0F70914B0F27
:105990002091B7053091B805621B730B882777FDFE
:1059A0008095982F0E947F218FE698E10E94B10D8B
:1059B0000E94720D08951F930E947718E0915B0C6E
:1059C000F0915C0C80818D3081F50E94C412182FFB
:1059D0008D3528F48A3558F48535C9F405C08F3FD4
:1059E000B1F488E599E152C081E499E14FC08BE2BE
:1059F00099E10E94B10D1A3511F480E305C01B3501
:105A000011F481E301C082E30E94D00D0AC082E15B
:105A100099E10E94B10D612F70E080E090E00E945A
:105A20007F218EE20E94D00D33C08DEF92E00E9464
:105A30006B19892B19F08FEF90E023C081E093E080
:105A40000E946B19892B19F085E590E01AC084E05B
:105A500093E00E946B19892B19F08AE590E011C040
:105A600088E093E00E946B19892B19F08BE590E098
:105A700008C08CE093E00E946B19892B29F08CE51B
:105A800090E00E94DC1604C085ED98E10E94B10D03
:105A90001F910895089508950895089584EE9CE057
:105AA0006BE774E04CE30E94FE1780EE9CE069E92E
:105AB00075E04EE10E94041810926C051092510698
:105AC00010925A0C08950E94E20C1092510F1092FD
:105AD000500F1092BE050895FB01E80FF91FDB017E
:105AE00002C081918D938091720590917305E817A2
:105AF000F907B8F3B0937305A093720508959C015C
:105B0000E091560CF091570C808191818217930798
:105B100014F0CF0108958281E80FF11DF5CFE091D7
:105B2000560CF091570C409172055091730520E08E
:105B300030E00BC0208131812115310519F420E0BE
:105B400030E006C08281E80FF11DE417F50791F7F8
:105B5000C90108959C018091500F9091510F8217B7
:105B60009307A0F1E091560CF091570CDF014D9195
:105B70005D914217530724F04217530739F507C0C8
:105B80008281E82FF0E03297EA0FFB1FEFCF8C9174
:105B9000DF01A80FB11D02C08D9181938091720524
:105BA00090917305A817B907B8F3F0937305E093C4
:105BB00072058091500F9091510F4817590731F499
:105BC0000E948F2D9093510F8093500F0895A091B4
:105BD0007205B0917305FD01E80FF91F8091440C27
:105BE0009091450C8E179F0720F489E08093460C16
:105BF0000895F0937305E09372056150704004C0FE
:105C00008C91808331971197A617B707C9F708952C
:105C1000DC0180915A0F282F30E088E59FE09093B7
:105C2000530C8093520C0CC0E091520CF091530C29
:105C300081918D93F093530CE093520C215030409E
:105C40002115310589F70895CF93DF93EC018091F9
:105C50005A0F90E0BE010E94E72D8091460C8823E8
:105C600019F4CE010E94082EDF91CF910895409142
:105C700072055091730580915A0F9A01280F311DBA
:105C80008091440C9091450C8217930780F0CA01D3
:105C90000E94082E20915A0F8091720590917305F1
:105CA000820F911D9093730580937205089589E08A
:105CB0008093460C0895CF93DF93EC018A81282FBF
:105CC00030E080915A0F281B31092115310501F16F
:105CD00037FF0CC088279927821B930BBE010E94B7
:105CE000E72D8091460C8823B1F412C0DE01A20F8B
:105CF000B31FFE0102C08D91819380917205909136
:105D00007305A817B907B8F3F0937305E09372050C
:105D1000CE010E94082EDF91CF910895CF93DF939B
:105D200081E08093430C88E59FE09093530C80932F
:105D3000520CC091580FD091590F8091500F9091F3
:105D4000510F8C179D0738F40E94372ED093510FB6
:105D5000C093500F18C0E091560CF091570C808101
:105D600091818C179D0724F0C817D90749F404C006
:105D70008281E80FF11DF3CFCF010E945B2E03C09B
:105D8000CF010E94242EDF91CF91089590E00197DA
:105D9000FC01EE0FFF1FE80FF91FEE0FFF1FEE0FC4
:105DA000FF1FE452F54F85919491009711F0FC018B
:105DB00009950895EF92FF920F931F93CF93DF936E
:105DC0002091E50C81E090E0821B9109880F991FDA
:105DD000880F991FC091E60CD091E70CC81BD90B16
:105DE000288139814A815B81CA01AA27BB27F90131
:105DF0000BB68BBF819190810BBE7C0100E010E05F
:105E00002E5F3F4F4F4F5F4FCA01AA27BB27F901B3
:105E10000BB68BBF219130810BBEC901A0E0B0E071
:105E2000DC01992788278E0D9F1DA01FB11F888335
:105E30009983AA83BB83DF91CF911F910F91FF902C
:105E4000EF900895CF93DF932091E50C81E090E0EF
:105E5000821B9109880F991F880F991FC091E60C2A
:105E6000D091E70CC81BD90B88819981AA81BB818D
:105E70009D0144275527FC010BB62BBF80810BBE2B
:105E800090E0A0E0B0E088839983AA83BB83DF9190
:105E9000CF910895CF93DF932091E50C81E090E0BE
:105EA000821B9109880F991F880F991FC091E60CDA
:105EB000D091E70CC81BD90B88819981AA81BB813D
:105EC0009D0144275527FC010BB62BBF8191908182
:105ED0000BBEA0E0B0E088839983AA83BB83DF91E7
:105EE000CF9108952091E50C81E090E0821B91090B
:105EF000880F991F880F991FE091E60CF091E70C2D
:105F0000E81BF90B80819181A281B38180959095E6
:105F1000A095B09580839183A283B3830895209147
:105F2000E50C81E090E0821B9109880F991F880F92
:105F3000991FE091E60CF091E70CE81BF90B8081CA
:105F40009181909581959F4FAA2797FDA095BA2F93
:105F500080839183A283B383089589E28093460C62
:105F600008956F927F928F929F92AF92BF92CF923D
:105F7000DF92EF92FF920F931F93CF93DF9384EE04
:105F80009CE068E30E943718AC01CB01DA015C01A8
:105F90006D012091E50C81E090E0821B9109880F52
:105FA000991F880F991FC091E60CD091E70CC81B70
:105FB000D90B288139814A815B81D7FE04C0EE2448
:105FC000FF24870126C039014A0171E0E72EF12C38
:105FD000012D112D19C0C50181709070892B41F0E0
:105FE000C801B7019301A4010E948E3E7B018C0180
:105FF000B301C4019301A4010E948E3E3B014C01F8
:10600000D594C794B794A794A114B104C104D10442
:1060100011F7E882F9820A831B83DF91CF911F91E8
:106020000F91FF90EF90DF90CF90BF90AF909F9037
:106030008F907F906F90089584EE9CE068E30E94BB
:1060400037184091E50C21E030E0241B3109220F84
:10605000331F220F331FE091E60CF091E70CE21B97
:10606000F30B20813181428153812617370748077E
:10607000590749F081E090E0A0E0B0E0808391838F
:10608000A283B3830895108211821282138208952D
:1060900084EE9CE068E30E9437184091E50C21E013
:1060A00030E0241B3109220F331F220F331FE091F0
:1060B000E60CF091E70CE21BF30B20813181428169
:1060C0005381261737074807590749F481E090E0C4
:1060D000A0E0B0E080839183A283B383089510820F
:1060E000118212821382089584EE9CE068E30E947C
:1060F00037184091E50C21E030E0241B3109220FD4
:10610000331F220F331FE091E60CF091E70CE21BE6
:10611000F30B2081318142815381261737074807CD
:1061200059074CF081E090E0A0E0B0E080839183DB
:10613000A283B3830895108211821282138208957C
:1061400084EE9CE068E30E9437184091E50C21E062
:1061500030E0241B3109220F331F220F331FE0913F
:10616000E60CF091E70CE21BF30B208131814281B8
:10617000538162177307840795074CF081E090E024
:10618000A0E0B0E080839183A283B383089510825E
:10619000118212821382089584EE9CE068E30E94CB
:1061A00037184091E50C21E030E0241B3109220F23
:1061B000331F220F331FE091E60CF091E70CE21B36
:1061C000F30B208131814281538162177307840769
:1061D00095074CF481E090E0A0E0B0E080839183EB
:1061E000A283B383089510821182128213820895CC
:1061F00084EE9CE068E30E9437184091E50C21E0B2
:1062000030E0241B3109220F331F220F331FE0918E
:10621000E60CF091E70CE21BF30B20813181428107
:10622000538126173707480759074CF481E090E05F
:10623000A0E0B0E080839183A283B38308951082AD
:1062400011821282138208950F931F9384EE9CE0B3
:1062500068E30E9437189B01AC016091E50C81E076
:1062600090E0861B9109880F991F880F991F009154
:10627000E60C1091E70C081B190BF8016081718185
:10628000828193810E948E3EF801608371838283B4
:1062900093831F910F9108950F931F9384EE9CE0B9
:1062A00068E30E9437189B01AC016091E50C81E026
:1062B00090E0861B9109880F991F880F991F009104
:1062C000E60C1091E70C081B190BF8016081718135
:1062D000828193810E94EF3EF80160837183828303
:1062E00093831F910F91089584EE9CE068E30E94D0
:1062F00037184091E50C21E030E0241B3109220FD2
:10630000331F220F331FE091E60CF091E70CE21BE4
:10631000F30B2081318142815381261B370B480BBF
:10632000590B2083318342835383089584EE9CE08C
:1063300068E30E9437184091E50C21E030E0241B0F
:106340003109220F331F220F331FE091E60CF09129
:10635000E70CE21BF30B2081318142815381260F30
:10636000371F481F591F2083318342835383089569
:1063700084EE9CE068E30E9437184091E50C21E030
:1063800030E0241B3109220F331F220F331FE0910D
:10639000E60CF091E70CE21BF30B20813181428186
:1063A0005381262337234823592320833183428373
:1063B0005383089584EE9CE068E30E94371840916F
:1063C000E50C21E030E0241B3109220F331F220F9E
:1063D000331FE091E60CF091E70CE21BF30B2081F8
:1063E000318142815381262B372B482B592B208317
:1063F000318342835383089584EE9CE068E30E94D6
:1064000037184091E50C21E030E0241B3109220FC0
:10641000331F220F331FE091E60CF091E70CE21BD3
:10642000F30B20813181428153812627372748276A
:1064300059272083318342835383089584EE9CE05F
:1064400068E30E943718CB010895CF92DF92EF9254
:10645000FF920F931F9384EE9CE068E30E9437182D
:106460006B017C01C114D104E104F104F9F0209125
:10647000E50C81E090E0821B9109880F991F880F3D
:10648000991F0091E60C1091E70C081B190BF801FD
:106490006081718182819381A70196010E94EF3E04
:1064A000F801208331834283538305C08AE18093BE
:1064B000460C0E94F9211F910F91FF90EF90DF9001
:1064C000CF9008950F931F93682F80EE9CE047E1D3
:1064D0000E941D183DC08091460C8823F1F5E09183
:1064E000E20CF091E30CE90FF11D42915291403121
:1064F000A1F1242F30E0207F3070852F90E0807F45
:106500009070821793074CF1413169F4503159F47E
:1065100080EE9CE068E30E940A1880EE9CE068E34D
:106520000E940A181AC080EE9CE068E30E940A18D4
:10653000082F80EE9CE068E30E940A18182F80EE76
:106540009CE0602F47E10E941D18812F0E94C62EFB
:106550009091E10C923008F0BECF1F910F910895F9
:10656000893328F4873360F4813141F409C08A33D8
:1065700039F08A3318F08A57863010F080E0089599
:1065800081E10E94623281E00895CF93DF938438E5
:1065900061F0853820F4833809F081C070C08439F7
:1065A00079F1843A09F07BC014C0E091520CF0916B
:1065B000530C818192813396F093530CE093520CEB
:1065C0000F960E94450DFC014081518162817381CB
:1065D0006CC0E091520CF091530C41815281638167
:1065E00074813596F093530CE093520C3597858166
:1065F0003696E80FF11DF093530CE093520C55C002
:10660000E091520CF091530C818192813396F0937A
:10661000530CE093520C0F960E94450DFC01C08173
:10662000D1818091520C9091530C01969093530C10
:106630008093520C0E945D338091520C9091530CC8
:1066400001969093530C8093520C84EE9CE068E387
:106650000E943718FB0188819981E817F90720F01B
:1066600089E18093460C26C0EE0FFF1FEE0FFF1F3F
:10667000EC0FFD1F428153816481758116C0E0914A
:10668000520CF091530C818192813396F093530C0C
:10669000E093520C0E94620EAB01BC0106C088E080
:1066A0008093460C0E94F92105C084EE9CE027E10E
:1066B0000E945718DF91CF9108951F9380E10E94A7
:1066C00062320E94D126E091520CF091530C8081ED
:1066D000803141F43196F093530CE093520C0E94B8
:1066E0005D3318C087FF07C00E94C5328091460CF9
:1066F000882339F319C00E940236182F8091460C66
:10670000882391F4812F0E94B032882369F4812F6D
:106710000E9462328091520C9091530C019690939A
:10672000530C8093520CCDCF1F910895EF92FF929E
:106730000F931F93CF93DF930E945D332091E50C5D
:1067400081E090E0821B9109880F991F880F991FA3
:10675000C091E60CD091E70CC81BD90BE880F980FA
:106760000A811B81E114F1040105110569F48EE42D
:1067700091E6ACEBB0E08093100390931103A093EB
:106780001203B093130328C060911003709111039A
:1067900080911203909113032DE036E649E150E019
:1067A0000E948E3E615A7C408149934C6093100355
:1067B000709311038093120390931303A801970120
:1067C0000E94CD3E9B01AC012F5F3F4F4F4F5F4F6B
:1067D000288339834A835B83DF91CF911F910F9187
:1067E000FF90EF900895AF92BF92CF92DF92EF9219
:1067F000FF920F931F930E945D332091E50C81E07F
:1068000090E0821B9109880F991F880F991FE091D2
:10681000E60CF091E70CE81BF90BA080B180C28078
:10682000D380E12CF12C012DA0E41A2F07C072E0D7
:1068300016950795F794E7947A95D1F7AE14BF04AF
:10684000C006D106A0F320E030E040E050E024C0D4
:10685000D801C701820F931FA41FB51FA816B90640
:10686000CA06DB0670F0A81AB90ACA0ADB0AD80100
:10687000C701880F991FAA1FBB1F280F391F4A1F66
:106880005B1F569547953795279582E01695079596
:10689000F794E7948A95D1F7E114F1040105110505
:1068A000B9F62A153B054C055D0520F42F5F3F4FD7
:1068B0004F4F5F4F20833183428353831F910F914A
:1068C000FF90EF90DF90CF90BF90AF9008951F930F
:1068D000DF93CF9300D000D0CDB7DEB7182F0E9442
:1068E0005D332091E50C81E090E0821B9109880FD7
:1068F000991F880F991FE091E60CF091E70CE81BB7
:10690000F90B6081718182819381123039F01430EA
:1069100071F0113099F40E94F2130BC00E94EC1236
:1069200069837A838B839C830E94720D0EC00E94C0
:10693000101369837A838B839C8307C083E08093E1
:10694000460C19821A821B821C8229813A814B8152
:106950005C816091E50C81E090E0861B9109880FD5
:10696000991F880F991FE091E60CF091E70CE81B46
:10697000F90B20833183428353830F900F900F9044
:106980000F90CF91DF911F91089584E00E946734AA
:10699000089582E00E946734089581E00E94673480
:1069A00008950E945D332091E50C81E090E0821B08
:1069B0009109880F991F880F991FE091E60CF091BB
:1069C000E70CE81BF90BA081B1818D919D910D9091
:1069D000BC91A02D80839183A283B38308950E94EC
:1069E0005D332091E50C81E090E0821B9109880FD6
:1069F000991F880F991FE091E60CF091E70CE81BB6
:106A0000F90BA081B1818D919C91A0E0B0E08083D1
:106A10009183A283B38308950E945D332091E50C96
:106A200081E090E0821B9109880F991F880F991FC0
:106A3000E091E60CF091E70CE81BF90BA081B18125
:106A40008C9190E0A0E0B0E080839183A283B38337
:106A500008950E945D3308950E945D332091E50CF6
:106A600081E090E0821B9109880F991F880F991F80
:106A7000E091E60CF091E70CE81BF90B8081918125
:106A8000A281B3810097A105B10529F4108211827A
:106A9000128213820895B7FF05C08FEF9FEFAFEF0B
:106AA000BFEF04C081E090E0A0E0B0E0808391837C
:106AB000A283B38308950E945D332091E50C81E0A9
:106AC00090E0821B9109880F991F880F991FE09110
:106AD000E60CF091E70CE81BF90B2081318137FFC0
:106AE00003C0309521953F4FC901AA2797FDA09576
:106AF000BA2F80839183A283B3830895CF93DF93CA
:106B0000843861F0853820F4833809F06DC05CC0AA
:106B10008439D1F0843A09F067C014C0E091520C76
:106B2000F091530C818192813396F093530CE09352
:106B3000520C0F960E94450DAC01662757FD6095DB
:106B4000762F58C08AE351C0E091520CF091530C5B
:106B5000818192813396F093530CE093520C0F96FF
:106B60000E94450DFC01C081D1818091520C909111
:106B7000530C01969093530C8093520C0E945D33FA
:106B80008091520C9091530C01969093530C8093EA
:106B9000520C84EE9CE068E30E943718888199814A
:106BA0006817790720F089E18093460C28C0229667
:106BB000660F771F660F771FC60FD71FAE016627B8
:106BC00057FD6095762F16C0E091520CF091530C52
:106BD000818192813396F093530CE093520C0E9482
:106BE0000D0DAB01BC0106C088E08093460C0E94ED
:106BF000F92105C084EE9CE027E10E945718DF913F
:106C0000CF910895863309F071C0E091520CF09154
:106C1000530C3196F093530CE093520C31978181D1
:106C20003396F093530CE093520C33978A30F1F182
:106C30008B3098F4853059F1863040F4833021F15F
:106C40008430F8F4823009F041C039C08730B9F19E
:106C5000873000F18930D1F520C08F3009F18031C3
:106C600038F48D3061F18E3050F58B3079F527C0D6
:106C7000813149F18131B8F08231D9F0833131F578
:106C80001BC00E945B3522C00E94F3331FC00E94CC
:106C900096331CC00E942C3519C00E940C3516C0BA
:106CA0000E94EF3413C00E94D13410C00E94CD3432
:106CB0000DC00E94C9340AC00E94C53407C089E2D1
:106CC0008093460C03C083810E947E358091520CD4
:106CD0009091530C01969093530C8093520C0E9408
:106CE000D126E091520CF091530C80810895E091EF
:106CF000520CF091530C8081E80FF11DF093530C6E
:106D0000E093520C0895E091520CF091530C808165
:106D1000E80FF11DF093530CE093520C0895A091ED
:106D2000520CB091530CFD012191F093530CE09360
:106D3000520C243951F411962D913C9112971396CF
:106D4000B093530CA093520C18C0223819F420E0D1
:106D500030E015C011968D919C911297FD013396EC
:106D6000233831F49C01F093530CE093520C07C08C
:106D7000F093530CE093520C9C01215F3F4FC901EB
:106D80000895E0915106EE2321F48DE18093460CA5
:106D90000895E150E0935106F0E0EE0FFF1FE85236
:106DA000F04F808191819093530C8093520C089501
:106DB00008950895CF93DF93E0915A0CEE2331F4B8
:106DC0008FE18093460C0E94F92124C0C091520C9F
:106DD000D091530CF0E0EE0FFF1FEA58FA4F80817C
:106DE00091819093530C8093520C0E945D3384EEFA
:106DF0009CE068E30E9437186115710581059105D3
:106E000049F4D093530CC093520C80915A0C81508A
:106E100080935A0CDF91CF910895CF93DF930E9416
:106E2000D126C091520CD091530C8091BE0588237D
:106E300051F0809172059091730501979093530CD6
:106E40008093520C06C02396D093530CC093520CDF
:106E500023970E94D12620915106203121F48CE104
:106E60008093460C13C0E22FF0E0EE0FFF1FE852B4
:106E7000F04F8091520C9091530C918380832F5F3F
:106E800020935106D093530CC093520CDF91CF91B5
:106E900008950E94720D81E08093430C10925E0C65
:106EA00010925D0C809172059091730501979093FB
:106EB000530C8093520C0895CF93DF9320915A0C7A
:106EC000203131F48EE18093460C0E94F92141C0BB
:106ED000E22FF0E0EE0FFF1FE858FA4F8091520CBE
:106EE0009091530C918380832F5F20935A0CC1E0C3
:106EF000D0E0E0917605F0917705F093530CE093A4
:106F0000520C309731F18091720590917305E8171A
:106F1000F90719F40E9449371CC082819F01280F8C
:106F2000311D30937705209376053396F093530CFB
:106F3000E093520C0E94D126E091520CF091530C38
:106F4000E081E93111F42196D4CFEA3191F621970D
:106F500081F6DF91CF9108958FE699E10E94B10DFE
:106F600060915D0C70915E0C80E090E00E947F214A
:106F70001092430C80917605909177059093570F6E
:106F80008093560F10925E0C10925D0C80917205EA
:106F90009091730501979093530C8093520C089530
:106FA0000E94D126E091520CF091530C2181328144
:106FB0003396F093530CE093520C5091BE05552339
:106FC00041F08091720590917305909377058093BD
:106FD0007605E0917605F0917705609172057091E4
:106FE0007305E617F70721F4E091560CF091570C62
:106FF000808191812817390720F4E091560CF09197
:10700000570C8081918182179307B1F4F093530C50
:10701000E093520C552341F01092BE0581E080931D
:107020004E060E94B42808953396F093530CE093D3
:10703000520C0E94D126089542812817390728F062
:10704000E40FF11DE617F707E1F68BE18093460C9C
:107050000895AF92BF92CF92DF92EF92FF920F937B
:107060001F93CF93DF93E091520CF091530C10815A
:10707000103731F0133721F0143711F000E00DC054
:107080003196F093530CE093520C0E94D126E0917C
:10709000520CF091530C012F10810E948F367C010D
:1070A000143919F0C0E0D0E034C08091520C9091B6
:1070B000530C01969093530C8093520C0E945D33B5
:1070C0008091520C9091530C01969093530C8093A5
:1070D000520C8091460C882309F082C0C7010E949F
:1070E000450DFC01C081D18184EE9CE068E30E94E3
:1070F0003718888199816817790720F089E1809392
:10710000460C6EC02296660F771F660F771FC60F5C
:10711000D71F0E94D1268091520C9091530C01965A
:107120009093530C8093520C0E945D338091460CD7
:10713000882309F055C084EE9CE068E30E9437186C
:107140005B016C01133831F4C701B601A5010E943F
:10715000210E46C0143929F4688379838A839B837E
:107160003FC0C7010E94450DFC010023D9F02081DA
:10717000318142815381003749F4CA01AA27BB27D4
:10718000F9010BB68BBFA0820BBE2AC0043779F47D
:10719000CA01AA27BB27F9010BB68BBFA192B08207
:1071A0000BBE1EC09C01442737FD4095542FCA01D9
:1071B000AA27BB27F9010BB68BBFA192B0820BBEE9
:1071C0002E5F3F4F4F4F5F4F7A0100271127C601B7
:1071D000AA27BB27F9010BB6EBBE819390830BBEA8
:1071E000DF91CF911F910F91FF90EF90DF90CF90A3
:1071F000BF90AF9008958FEF80936B050895109224
:107200006B05089508958091520C9091530C03964C
:107210009093530C8093520C0E945D338091520CDA
:107220009091530C01969093530C8093520C0895B7
:107230001F93182F82958F708A3008F0895F805DC8
:107240000E94D00D812F8F708A3008F0895F805D99
:107250000E94D00D1F910895EF92FF920F931F93FC
:107260000E94033984EE9CE068E30E9437187B019A
:107270008C01892F9927AA27BB270E941839C8019A
:10728000AA27BB270E941839BB27A12F902F8F2D2B
:107290000E9418398E2D0E9418391F910F91FF906E
:1072A000EF900895EF92FF920F931F930E9403397E
:1072B00084EE9CE068E30E9437187B018C01BB27B9
:1072C000A92F982F872F0E9418398E2D0E941839C8
:1072D0001F910F91FF90EF9008950E94033984EE63
:1072E0009CE068E30E943718862F0E9418390895A1
:1072F0000E94033984EE9CE068E30E943718862FD1
:107300000E94D00D08950E94033984EE9CE068E34A
:107310000E94371889E00E94D00D0895EF92FF92E5
:107320000F931F930E94D126E091520CF091530CC1
:10733000E08110E07BC0EB37B1F1EC3720F4E633AD
:1073400009F05FC03BC0EC3759F1E23A09F059C08F
:10735000E091520CF091530C6181E62EFF2400E085
:1073600010E08EEF9FEFAFEFBFEFE80EF91E0A1FA0
:107370001B1F3396F093530CE093520CCF01B701CF
:107380000E94D83CB7016F5F7F4F8091520C909163
:10739000530C860F971F9093530C8093520C23C06D
:1073A00089E00E94D00D8091520C9091530C01966F
:1073B0009093530C8093520C11E031C0E091520C29
:1073C000F091530C81818B3099F08C3028F482300D
:1073D00061F08730B1F405C08D3069F08E3089F4EA
:1073E0000DC00E94833910E01AC00E94783928C06D
:1073F0000E942C3925C00E946D3922C00E9452394A
:107400001FC00E945D338091460C8823E9F484EE0E
:107410009CE068E30E9437180E947F2111C00E94FF
:10742000D126E091520CF091530CE081ED3719F028
:10743000EA3709F080CF112339F40E94720D04C09D
:1074400080E20E94D00DCFCF1F910F91FF90EF905F
:107450000895EF92FF920F931F93CF93DF93E090E5
:10746000B705F090B8050E94D126E091520CF0913A
:10747000530C808184FD02C081E22FC08181928102
:107480000F960E94450DEC018091520C9091530C87
:1074900004969093530C8093520C0E945D3380911C
:1074A000520C9091530C01969093530C8093520C74
:1074B00088819981AA81BB810097A105B10509F056
:1074C00047C00091B7051091B80584EE9CE068E3D1
:1074D0000E94371877FF04C087E28093460C47C0AC
:1074E0004091B7055091B805198308831B821A8211
:1074F0006F5F7F4FF801718360834E5F5F4FCB01F9
:10750000880F991F880F991F840F951F4250504074
:107510009093B8058093B70520914A0F30914B0F97
:107520002817390720F0FA0180E090E00EC089E0CA
:107530008093460CF092B805E092B70518C012820D
:107540001382148215820196349686179707B8F332
:107550000E94D126E091520CF091530C80818D371E
:1075600031F03196F093530CE093520C78CFDF91C9
:10757000CF911F910F91FF90EF9008950895089576
:107580000895089508950895089508950895089513
:1075900008958091BE05882329F083E38093460CEB
:1075A0000E94F9210895CF93DF93C091520CD0919E
:1075B000530C8091560C9091570C9093530C8093E0
:1075C000520C90935F0680935E06E091520CF0910E
:1075D000530C82819F01280F311D30935F06209349
:1075E0005E063396F093530CE093520C0E94D12622
:1075F000E091520CF091530C80818C3051F4329612
:10760000F0935F06E0935E06D093530CC093520C48
:107610001AC020915E0630915F06809172059091AC
:1076200073052817390751F4D093530CC093520CAB
:1076300086E28093460C0E94F92105C03093530CDA
:107640002093520CC2CFDF91CF910895CF93DF9357
:10765000C091520CD091530C80915E0690915F06C0
:107660009093530C8093520C8091520C9091530C38
:1076700003969093530C8093520C0E94D126E09174
:10768000520CF091530C80818C3051F43396F0936E
:107690005F06E0935E06D093530CC093520C1BC060
:1076A000E0915E06F0915F068091720590917305FE
:1076B000E817F90741F4D093530CC093520C86E2BB
:1076C0008093460C08C08281E80FF11DF0935F069D
:1076D000E0935E06C9CFDF91CF910895CF92DF92FC
:1076E000EF92FF920F931F930E94D1260E948F3634
:1076F0008C010E94D40DC82EC8010E94450DFC01CA
:10770000DD24EE24FF24C082D182E282F3821F9125
:107710000F91FF90EF90DF90CF900895CF93DF937C
:107720000E94D1260E948F369C0190916C058EE0BC
:10773000989FE0011124CD54DA4F88819981281750
:10774000390731F084E28093460C0E94F92145C04C
:10775000C9010E94450DFC01208131814281538184
:107760008A819B81AC81BD81280F391F4A1F5B1F15
:1077700020833183428353838A819B81AC81BD8185
:10778000B7FF0AC08E819F81A885B9852817390760
:107790004A075B07B4F40DC00097A105B10589F055
:1077A0008E819F81A885B98582179307A407B507A5
:1077B00044F480916C05815080936C050E94D12621
:1077C0000CC08A859B859093530C8093520C8C85BA
:1077D0009D8590935E0C80935D0CDF91CF91089511
:1077E000DF92EF92FF920F931F93D82E8091520C4D
:1077F0009091530C01969093530C8093520C0E94DD
:10780000D1260E945D330E94D1268091520C909126
:10781000530C01969093530C8093520C0E94D126E6
:107820008091520C9091530C01969093530C80933D
:10783000520C0E945D3384EE9CE068E30E9437188E
:107840007B018C0184EE9CE068E30E94371822E003
:10785000D216A1F034E0D316F9F041E0D41611F5B8
:1078600080E090E02FEF30E040E050E0E222F322B1
:10787000042315234E2D0E948E1714C080E090E043
:107880002FEF3FEF40E050E0E222F32204231523E4
:10789000A7010E944D1706C080E090E0A801970163
:1078A0000E9466171F910F91FF90EF90DF9008954F
:1078B00084E00E94F03B089582E00E94F03B08952E
:1078C00081E00E94F03B08950E945D330E94D12622
:1078D0008091520C9091530C01969093530C80938D
:1078E000520C0E94D12684EE9CE068E30E94371877
:1078F0009B01AC018091460C8823C1F5E091520CAC
:10790000F091530C232B31F08081883A79F50E9455
:10791000D03708958081883A79F43396F093530CE8
:10792000E093520C0E94D126E091520CF091530C3E
:1079300080818933D9F40AC08091760590917705CA
:1079400001979093530C8093520C08953196F093C5
:10795000530CE093520C0E94D126E091520CF0910E
:10796000530C8081883A11F40E94D03708951F93F8
:10797000E0915B0CF0915C0C80818D3211F010E095
:1079800006C03196F0935C0CE0935B0C11E00E9412
:10799000AA1E9B01AC01112339F0509540953095FA
:1079A00021953F4F4F4F5F4FB901CA011F91089575
:1079B0000F931F93CF93DF938C01EB0106C0F80167
:1079C00081918F010E947B0D21972097C1F7DF9154
:1079D000CF911F910F910895EF92FF920F931F93F4
:1079E000E0915B0CF0915C0C8081843241F4319623
:1079F000F0935C0CE0935B0C0E944E1F02C00E944F
:107A0000B73C7B018C010E947718E0915B0CF091F0
:107A10005C0C80818D3071F08C3231F43196F093B2
:107A20005C0CE0935B0C06C085E18093460C0E94E1
:107A3000F92109C00E948F360E94450DFC01E082A9
:107A4000F182028313831F910F91FF90EF900895AD
:107A50000E947718E0915B0CF0915C0C80818D3076
:107A6000C9F00E94EC3C8091460C882399F40E9456
:107A7000D126E091520CF091530C80818D3769F042
:107A80008A3759F03196F093530CE093520C0E94D0
:107A9000D126DECF21E030E002C020E030E0C90195
:107AA000089580915E0690915F06892B21F40E94D3
:107AB000D33A0E94263B80915E0690915F06909398
:107AC0005C0C80935B0C0E94D1260E94283D209183
:107AD0005B0C30915C0C019769F42E5F3F4F309343
:107AE0005F0620935E060E94263B8091460C882309
:107AF00011F304C030935F0620935E060895EF9261
:107B0000FF920F931F930E94D126E091520CF091A7
:107B1000530C8081823A01F5018110E0025010403F
:107B200083E0E82EF12CEE0EFF1EC701B8010E9483
:107B3000D83C0F5F1F4FE00EF11EF092530CE09205
:107B4000520C0E94D1268091520C9091530C0196B8
:107B50009093530C8093520C0E94D1268FE30E9485
:107B6000D00D80E20E94D00D0E94D71A0E94720DA3
:107B70000E941927882321F40E94283D892B71F740
:107B80001092F80F1F910F91FF90EF9008950F93AF
:107B90001F9380916C058A3031F483E28093460C08
:107BA0000E94F921B8C00E94D1260091520C109178
:107BB000530C0E948F3640916C05242F30E0220F29
:107BC000331FF90173E0EE0FFF1F7A95E1F7E21B17
:107BD000F30BEF53FA4F91838083842F90E0880F4B
:107BE000991FFC0153E0EE0FFF1F5A95E1F7E81BC8
:107BF000F90BEF53FA4F80915D0C90915E0C9587D5
:107C000084871093530C0093520C0E9429380E94D1
:107C1000D1268091520C9091530C01969093530C65
:107C20008093520C0E94D1260E945D3310916C0506
:107C300084EE9CE068E30E943718212F30E0220F89
:107C4000331FF90103E0EE0FFF1F0A95E1F7E21B76
:107C5000F30BEF53FA4F6683778380879187809188
:107C60006C0590E0FC0113E0EE0FFF1F1A95E1F7A1
:107C7000E81BF90BEE0FFF1FED53FA4F81E090E088
:107C8000A0E0B0E080839183A283B3830E94D126D9
:107C9000E091520CF091530C80818A3319F53196A2
:107CA000F093530CE093520C0E94D1260E945D3356
:107CB00000916C0510E084EE9CE068E30E943718A8
:107CC000F801A3E0EE0FFF1FAA95E1F7E01BF10B0F
:107CD000EE0FFF1FED53FA4F60837183828393830E
:107CE0000E94D12620916C05822F90E0880F991F69
:107CF000FC0133E0EE0FFF1F3A95E1F7E81BF90BAB
:107D0000EF53FA4F8091520C9091530C93878287D6
:107D10002F5F20936C051F910F910895629FD001F2
:107D2000739FF001829FE00DF11D649FE00DF11D36
:107D3000929FF00D839FF00D749FF00D659FF00DE5
:107D40009927729FB00DE11DF91F639FB00DE11DD2
:107D5000F91FBD01CF0111240895991B79E004C0DA
:107D6000991F961708F0961B881F7A95C9F780957A
:107D70000895AA1BBB1B51E107C0AA1FBB1FA61772
:107D8000B70710F0A61BB70B881F991F5A95A9F7C4
:107D900080959095BC01CD010895A1E21A2EAA1BF1
:107DA000BB1BFD010DC0AA1FBB1FEE1FFF1FA217AB
:107DB000B307E407F50720F0A21BB30BE40BF50BA8
:107DC000661F771F881F991F1A9469F76095709531
:107DD000809590959B01AC01BD01CF01089597FB63
:107DE000092E05260ED057FD04D0D7DF0AD0001C7F
:107DF00038F450954095309521953F4F4F4F5F4F48
:107E00000895F6F790958095709561957F4F8F4F07
:107E10009F4F089585FD59C08062911156C08156CB
:107E20008A51E0F70895911150C080538A5028F08C
:107E3000865C806281568650B8F708959111089546
:107E400081548A5108F4805E855A089591110895ED
:107E500081568A5108F4805285580895FB01DC014F
:107E600005900D920020E1F70895FC010590002097
:107E7000E9F7809590958E0F9F1F0895FB01DC0117
:107E80000D900020E9F7119701900D920020E1F785
:107E90000895FB01DC0101900D920020E1F70895A7
:107EA000E199FECF9FBB8EBBE09A99278DB30895D1
:107EB000262FE199FECF9FBB8EBB2DBB0FB6F8944A
:107EC000E29AE19A0FBE01960895992788270895AE
:047ED000F894FFCF54
:107ED400010102014201430183018401646174616F
:107EE400006C6574007265616400726573746F720E
:107EF4006500676F73756200676F746F006F6E0063
:107F040072657475726E00696600696E70757400CE
:107F14007072696E7400666F72006E6578740073B7
:107F2400746F7000656E64776800656E64007265D6
:107F34006D0064696D0074726F6E0074726F6666B2
:107F4400007768696C650065657031360065657039
:107F540033320065657000696E62797465003F00B4
:107F64002700656C7365003C3D003E3D003C3E00CF
:107F74003C003E003D00414E44004F5200454F52EC
:107F8400002B002D002A002F006D6F64005E00405E
:107F94003136004033320040006E6F7400746F005D
:107FA40053544550007468656E00656C73650047F2
:107FB4004F544F00474F53554200434852240061E9
:107FC4006273007371727400524E440053474E0042
:107FD4005441420068657834006865783200686509
:107FE40078007065656B3136007065656B333200FF
:107FF4007065656B0061646472006565703136009C
:108004006565703332006565700074696D652400C0
:10801400706F727473004C697374206F6620706F94
:10802400727473202D2D00200076617273004C69E8
:108034007374206F66207661726961626C65732067
:108044002D2D00202020200028002900202000665B
:10805400696C657300556E6B6E6F776E204C495377
:108064005420746F7069632E202054727920276C19
:1080740069737420706F72747327206F7220276C79
:10808400697374207661727327206F7220276C697C
:1080940073742066696C6573272E006D6F6E006CB7
:1080A4006973740072756E006E657700636F6E7429
:1080B40000636C6561720066726565006C6F616473
:1080C4000073617665006175746F7374006F666622
:1080D40000656500666C3000666C3100666C3200C9
:0480E4004E61BC002D
:020000021000EC
:10FC0000AF92BF92CF92DF92EF92FF920F931F932A
:10FC1000CF93DF937B018C016A01AFB6F894E19931
:10FC2000FECF8091680080FDFCCF83E0F701009358
:10FC30005B0080936800E8958091680080FDFCCFB0
:10FC400040E050E060E070E0BB24B394F6018081B6
:10FC5000D181C0E09E01280F311D82E090E0C80EE6
:10FC6000D91EDB01CA018E0D9F1DA01FB11F090106
:10FC7000FC01A0935B00B0926800E89511244E5FF0
:10FC80005F4F6F4F7F4F403091E0590790E0690719
:10FC900090E07907D9F685E0F70100935B00809347
:10FCA0006800E8958091680080FDFCCF81E1809339
:10FCB0006800E895AFBEDF91CF911F910F91FF9043
:0CFCC000EF90DF90CF90BF90AF900895C0
:00000001FF
